:10000000004000204D610000A5610000215D00005E
:10001000A5610000A5610000A561000000000000CE
:10002000000000000000000000000000A5610000CA
:10003000A561000000000000A5610000A5610000AE
:10004000A5610000A5610000A5610000A561000098
:10005000ED45000031460000A5610000A5610000EB
:10006000754600008D470000A5610000A5610000F5
:10007000A12C0000E52B0000A5610000A561000097
:10008000A5610000A5610000A5610000A561000058
:10009000A5610000E939000075440000A561000079
:1000A00000000000A5610000A5610000A56100003E
:1000B000A56100004D480000A5610000A561000099
:1000C0000448054B10B5834203D0044B002B00D0ED
:1000D000984710BD940700209407002000000000FE
:1000E00006480749091A8B10C90FC91810B54910DD
:1000F00003D0044B002B00D0984710BD940700207C
:10010000940700200000000010B5074C2378002B56
:1001100009D1FFF7D5FF054B002B02D0044800E0C2
:1001200000BF0123237010BD9407002000000000D1
:10013000ECAB0000054B10B5002B03D0044905487B
:1001400000E000BFFFF7CCFF10BDC046000000007C
:1001500098070020ECAB0000402292029A1A9246C7
:100160007047C046174B002B00D1134B9D46FFF73D
:10017000F3FF00218B460F461348144A121A08F069
:10018000A7FF0E4B002B00D098470D4B002B00D043
:1001900098470020002104000D000D48002802D0DF
:1001A0000C4809F06FF909F02DF82000290005F03E
:1001B00055F908F03BFDC0460000080000000000B3
:1001C000000000000040002094070020D014002010
:1001D0008594000095A00000F0B52A4A2A4B1278B9
:1001E0008BB01A706822294E00233500310001922D
:1001F000274A38350692274A2C310792264A00951D
:100200000892264A0992069A2548D25A0A70079AF5
:10021000D25ACA70089AD25A8A71099AD25A4A7224
:10022000019AB4189A00101805901E4810180490EE
:100230001D48101803901D481218029200220098C1
:10024000059FBF5A3D0A0570049D4770AF5A0230A2
:100250003D0A8575039DC775AF5A029D2770AF5A39
:10026000023227730134082AEAD1009A0233083295
:100270000092019A013104320192062BC3D10BB0D6
:10028000F0BDC046D6000020460800201B08002014
:10029000EA000020E4000020DE000020D80000205A
:1002A00038010020F000002020010020080100207B
:1002B000F8B508F0C7FB864A864B0D00040008F02D
:1002C000D1F8854A854B07F0A1F9854A06000F0051
:1002D000844B2900200008F0C5F82B00220008F00C
:1002E000C1F802000B003000390007F08FF97E4A98
:1002F00006000F007D4B2900200008F0B3F82B000A
:10030000220008F0AFF82B00220008F0ABF8020042
:100310000B003000390007F079F9754A06000F002C
:10032000744B2900200008F09DF82B00220008F0F3
:1003300099F82B00220008F095F82B00220008F015
:1003400091F802000B003000390007F05FF96A4AAB
:1003500006000F00694B2900200008F083F82B00ED
:10036000220008F07FF82B00220008F07BF82B0019
:10037000220008F077F82B00220008F073F8020042
:100380000B003000390007F041F95D4A06000F000C
:100390005C4B2900200008F065F82B00220008F0D3
:1003A00061F82B00220008F05DF82B00220008F015
:1003B00059F82B00220008F055F82B00220008F015
:1003C00051F802000B003000390007F01FF94E4AC7
:1003D00006000F004D4B2900200008F043F82B00C9
:1003E000220008F03FF82B00220008F03BF82B0019
:1003F000220008F037F82B00220008F033F82B0019
:10040000220008F02FF82B00220008F02BF8020041
:100410000B003000390007F0F9F83D4A06000F00E4
:100420003C4B2900200008F01DF82B00220008F0AA
:1004300019F82B00220008F015F82B00220008F014
:1004400011F82B00220008F00DF82B00220008F014
:1004500009F82B00220008F005F82B00220008F014
:1004600001F802000B003000390007F0CFF82A4AEB
:1004700006000F00294B2900200007F0F3FF2B0096
:10048000220007F0EFFF2B00220007F0EBFF2B000C
:10049000220007F0E7FF2B00220007F0E3FF2B000C
:1004A000220007F0DFFF2B00220007F0DBFF2B000C
:1004B000220007F0D7FF2B00220007F0D3FF020035
:1004C0000B003000390007F0A1F808F001FBF8BD7F
:1004D000C15609167F6A8B407652FCC1378F9F3F09
:1004E000899854651ED3A8C0E5BB529EECF4B54074
:1004F0009EC6C56A10EDB6C0E1070862CEE8AD4001
:1005000046962FDC0FA298C049282721BBDF7840F0
:1005100001B8484741184CC018EC0EDB17280B40B7
:1005200010B507F031F808F08DFA044A044B07F0D3
:1005300099FF08F0CDFAFFF7BBFE10BDB4D934E740
:100540000C684A3FF0B50C0085B0051C2422081D3C
:1005500008F03CFD23002833039300230293164B3D
:1005600025600093154B019326680199301C05F016
:10057000DFFF351C002800D1019D0099301C01953A
:1005800005F0C2FF371C002800D1009F0298311CE3
:10059000009705F0EFFF039B04340290A342E3D1E0
:1005A000291C06F03FFD391C06F03CFDF8218905A9
:1005B00006F0EEFB05B0F0BD00401C4600401CC636
:1005C00070B512220C000500881C08F0FFFC00200A
:1005D00026000300210025800A4C14360A88151CC9
:1005E0009A4200D21D1CABB2151CA24200D9251C98
:1005F0000231ACB280188E42F0D11B19C01AC0086B
:1006000080B270BD10270000F8B53C4B3C4C1A7806
:10061000012A59D100221A7020693A4D00053A4941
:10062000000D2880FFF7CCFF384B1880606800056C
:10063000000DFFF775FF0021061C05F05BFF002889
:1006400009D0301C08F0FEF9314A324B07F00AFF9E
:1006500008F03EFA061C301C06F02EFF03002E4E5A
:10066000283337787D2B35D9022364201F432B4B49
:1006700037701860A068AF260005000D06F084FFF3
:1006800008F0E0F9264A274B07F0D4FB0022264B5E
:1006900007F0E8FE08F09EF9244F301A3880E06831
:1006A0000005000D288006F06FFF08F0CBF91C4A0A
:1006B0001C4B07F0BFFB00221B4B07F0D3FE08F0DA
:1006C00089F91B4D361A2E808023A26C1B0113431F
:1006D000A364F8BD06F010FF1649FFF733FF0223AD
:1006E0009F4306F0E9FE0300143302DA142040426F
:1006F000BDE75528BBDD5520B9E7C04604110020F1
:1007000000000E40FE070020B4070020FC07002078
:10071000CDCCCCCCCCCCF03FB3070020F8070020E8
:10072000E17A14AE476110400000D03FF20700208C
:10073000F0070020C8070020F0B514228BB000217C
:10074000CA4808F0C5FC14220021C94808F0C0FCC2
:1007500014220021C74808F0BBFC0025C64CE8B2B3
:100760006119013505F0A8F8802DF7D1627823785A
:100770001202A1781343E278090412060B431343D3
:10078000BE4A934200D0F9E1A27ABD4B1A70E27AD8
:10079000BC4B1A70227BBC4B1A70627BBB4B1A702D
:1007A000A27BBB4B1A70E27BBA4B1A70227CBA4B0D
:1007B0001A70627CB94B1A70A27CB94B1A70E27C39
:1007C000B84B1A70227DB84B1A70627DB74B1A7005
:1007D000A27DB74B1A70E27DB64B1A70227EB64BE3
:1007E0001A70627EB54B1A70A27EB54B1A70E27E0B
:1007F000B44B1A70227FB44B1A70627FB34B1A70DD
:10080000A27FB34B1A70E27FB24B1A70621CD27F88
:10081000B14B1A70A21CD27FB04B1A70E31CDA7F66
:10082000231DDB7F1B021343AD4A5BBA1380631D9C
:10083000DA7FA31DDB7F1B021343AA4A5BBA138036
:10084000E31DDA7F23000833DB7F1B021343A64A34
:100850005BBA1380220028321278A44B1A7022004F
:1008600029321278A24B1A7022002A32A14B127838
:100870001A7023002B331B780393022B00D984E0DA
:100880002300383301930293183D0020631900932D
:10089000844604230100029A059003E03000049E80
:1008A0000597B44616780F00517836023143B942A5
:1008B0006BD9177E567E3F023E430496664564D947
:1008C000009F059E3F78B7425FD9009E367B8642E7
:1008D0005BD90098013B0130DBB202320090002B63
:1008E000DCD1029A043508320292742DCDD1824AAD
:1008F00003991170682221000092804A2C310692DF
:100900007F4A07927F4A08927F4A09920A7806989E
:10091000C252CA780798C2528A790898C2524A7A53
:100920000998C252009A7948A5189A0010180290A6
:1009300077481018059077481018049076481218D8
:1009400003920022019807783F023E004778023068
:100950003743029EB752877D3E02C77D3743059ECF
:10096000B7522F78049E0135B752EF7A039EB752E3
:100970000232082AE7D1019A023308320192009A22
:10098000013104320092062BC0D13D4A634B1278EC
:100990000A241A703B4A624B12781A703A4A614B29
:1009A00012781A70394A604B12781A70384A5F4BC5
:1009B00012781A70374A5E4B12781A70364A5D4BBD
:1009C00012781A70354A5C4B12781A705B4B344AB5
:1009D00012781A70334A5A4B12781A70324A594BAD
:1009E00012781A70314A584B12781A70304A574BA5
:1009F00012781A702F4A564B12781A702E4A554B9D
:100A000012781A702D4A544B12781A70534B2C4A94
:100A100012781A702B4A524B12781A702A4A514B8C
:100A200012781A70294A504B12781A70284A4F4B84
:100A300012781A70274A4E4B12781A70264A4D4B7C
:100A400012781A70254A4C4B12781A7000F060FD2B
:100A5000642003F068FD013CFFF7D6FDA4B214202A
:100A600003F061FD002CF6D10BB0F0BD1D1000208D
:100A70009A1000205E1000201B080020AA55AA55DD
:100A80007B0900207A0900207909002078090020DC
:100A900077090020760900207509002074090020DC
:100AA00073090020720900207109002070090020DC
:100AB0006F0900206E0900206D0900206C090020DC
:100AC0006B0900206A0900206909002068090020DC
:100AD00067090020660900206509002064090020DC
:100AE000F8100020F6100020F4100020B2070020BB
:100AF000B1070020B0070020D6000020EA00002047
:100B0000E4000020DE000020D80000203801002092
:100B1000F00000202001002008010020180800201B
:100B200017080020160800201508002014080020CF
:100B300013080020120800201108002010080020CF
:100B40000F0800200E0800200D0800200C080020CF
:100B50000B0800200A0800200908002008080020CF
:100B600007080020060800200508002004080020CF
:100B7000030800200208002001080020AA233820D2
:100B80002370A3704E4B462218703F204D4B5626C3
:100B900018704D4B48251A7041224C4B55271E703A
:100BA0004B4B4E261A7050224A4B67701D704A4BB1
:100BB00000251E70494B39261A704322484BE770B6
:100BC0001A70484B38211A70474B1A70474B1A70ED
:100BD000474B1E704626474B1870474BA1721E703C
:100BE000464B474E1F70474B0E311D70464B2173CD
:100BF0001D70464B10311D70454B61731D704B23AA
:100C00003370444E15393370434EA1733370434EE5
:100C100007313370424EE072B4463580414E358024
:100C20000096414E3580E173A274E27422756275BC
:100C300006310A3A2174A27502310D3261742276AE
:100C4000A11C621CD377A377E377CB7763461B881D
:100C5000E21C1B0AD37763461A88231DDA77009BB0
:100C6000621D1B88E0751B0AD377009B67761A8884
:100C7000A31DDA773388E21D1B0AD377230032885D
:100C80000833DA772200A576E57625776577274B56
:100C900028321B781370264B1A78230029331A70D8
:100CA000244B2A341B782370FFF796FA224BE8B2C4
:100CB000595D013504F010FE802DF7D165E6C04680
:100CC0007B0900207A09002079090020780900209A
:100CD000770900207609002075090020740900209A
:100CE000730900207209002071090020700900209A
:100CF0006F0900206E0900206D0900206C0900209A
:100D0000670900206B0900206A090020690900209A
:100D10006809002066090020650900206409002098
:100D2000F8100020F6100020F41000200011002020
:100D300003110020011100201B08002070B53F4B5B
:100D40003F4C1B78621CA3723E4BE11C1B780025B4
:100D5000E3723D4B1B7823733C4B1B7863733C4B16
:100D60001B78A3733B4B1B78E3733B4B1B782374BB
:100D70003A4B1B7863743A4B1B78A374394B1B783E
:100D8000E374394B1B782375384B1B786375384BEC
:100D90001B78A375374B1B78E375374B1B7823768D
:100DA000364B1B786376364B1B78A376354B1B7816
:100DB000E376354B1B782377344B1B786377344BC2
:100DC0001B78A377334B1B78E377334B1B78D377B0
:100DD000324BA21C1B78D377314A138812881B0A26
:100DE000CB77231DDA772F4A611D138812881B0ADF
:100DF000CB77A31DDA772C4AE11D138812881B0AD2
:100E0000CB7723000833DA772200284B28321B786F
:100E10001370274B1A78230029331A70254B1A7840
:100E200023002A331A70FFF7D7F9615DE8B2013564
:100E300004F052FD802DF8D170BDC0467B09002022
:100E40001B0800207A090020790900207809002079
:100E50007709002076090020750900207409002018
:100E60007309002072090020710900207009002018
:100E70006F0900206E0900206D0900206C09002018
:100E80006B0900206A090020690900206809002018
:100E90006709002066090020650900206409002018
:100EA000F8100020F6100020F4100020001100209F
:100EB00003110020011100200721114A13788B43F0
:100EC000104913700A88104B002A06D11A88002A8C
:100ED00003D11A8890B2002A0DD000220A80FA218C
:100EE00018880901884200D31A80084B084A1988DB
:100EF000914201D80120704700221A80FAE7C046CB
:100F000000080020F8100020F6100020F410002047
:100F10001F4E000000230E4A13700E4A13700E4A33
:100F200013600E4A13700E4A13700E4A13700E4A65
:100F300053709370D370137153719371012805D15D
:100F40000A4A13600A4A13700A4A13707047C0466F
:100F5000DB0F0020DA0F0020FC1000200111002020
:100F60000311002000110020530F0020F40E002078
:100F7000F30E0020F20E002030B5274A1378012826
:100F80000DD1062B28D9002313700122234B1A60A0
:100F90000023234A1360234A1360234A2CE0002BCA
:100FA0000FD0013BD8B21070072826D800231B4D64
:100FB0001B4C1C491C4A05F0F7F8E811171B2125AA
:100FC0002906072313700123144A154913600022D0
:100FD0000A6014490A60E0E70133E3E701232B606C
:100FE000236000230B6007E001202B602060F9E7FD
:100FF00001202B6020600860136030BD2B60012051
:101000002360F8E72B6023600123EBE72B6023606C
:101010000B600123F0E7C046F40900207042005045
:1010200074420050784200506042005030B5274A68
:10103000137801280DD1062B28D900231370012223
:10104000234B1A600023234A1360234A1360234A68
:101050002CE0002B0FD0013BD8B21070072826D807
:1010600000231B4D1B4C1C491C4A05F09DF8E81140
:10107000171B21252906072313700123144A15493C
:10108000136000220A6014490A60E0E70133E3E7D5
:1010900001232B60236000230B6007E001202B60FD
:1010A0002060F9E701202B6020600860136030BDEC
:1010B0002B6001202360F8E72B6023600123EBE71E
:1010C0002B6023600B600123F0E7C046F30900208A
:1010D0007C420050B8420050BC4200509842005040
:1010E00030B5274A137801280DD1062B28D90023C3
:1010F00013700122234B1A600023234A1360234AF2
:101100001360234A2CE0002B0FD0013BD8B21070A3
:10111000072826D800231B4D1B4C1C491C4A05F0F0
:1011200043F8E811171B2125290607231370012313
:10113000144A1549136000220A6014490A60E0E766
:101140000133E3E701232B60236000230B6007E0FA
:1011500001202B602060F9E701202B6020600860EF
:10116000136030BD2B6001202360F8E72B60236003
:101170000123EBE72B6023600B600123F0E7C046FF
:10118000F209002018420050384200503C42005002
:10119000A042005030B5274A137801280DD1062B04
:1011A00028D9002313700122234B1A600023234AFD
:1011B0001360234A1360234A2CE0002B0FD0013B1D
:1011C000D8B21070072826D800231B4D1B4C1C4991
:1011D0001C4A04F0E9FFE811171B21252906072303
:1011E00013700123144A1549136000220A60144940
:1011F0000A60E0E70133E3E701232B60236000236B
:101200000B6007E001202B602060F9E701202B60D4
:1012100020600860136030BD2B6001202360F8E778
:101220002B6023600123EBE72B6023600B6001231D
:10123000F0E7C046F1090020A4420050A842005047
:10124000AC4200506442005030B5274A1378012860
:101250000DD1062B28D9002313700122234B1A60CD
:101260000023234A1360234A1360234A2CE0002BF7
:101270000FD0013BD8B21070072826D800231B4D91
:101280001B4C1C491C4A04F08FFFE811171B212539
:101290002906072313700123144A154913600022FD
:1012A0000A6014490A60E0E70133E3E701232B6099
:1012B000236000230B6007E001202B602060F9E72A
:1012C00001202B6020600860136030BD2B6001207E
:1012D0002360F8E72B6023600123EBE72B6023609A
:1012E0000B600123F0E7C046F0090020684200507F
:1012F000884200508C420050FC42005030B5274AD2
:10130000137801280DD1062B28D900231370012250
:10131000234B1A600023234A1360234A1360234A95
:101320002CE0002B0FD0013BD8B21070072826D834
:1013300000231B4D1B4C1C491C4A04F035FFE811CF
:10134000171B21252906072313700123144A154969
:10135000136000220A6014490A60E0E70133E3E702
:1013600001232B60236000230B6007E001202B602A
:101370002060F9E701202B6020600860136030BD19
:101380002B6001202360F8E72B6023600123EBE74B
:101390002B6023600B600123F0E7C046EF090020BB
:1013A000F8420050DC420050D84200504C420050FD
:1013B0000023044A1360044A1360044A1360044A79
:1013C00013607047704200507442005078420050E1
:1013D000604200500023044A1360044A1360044A28
:1013E0001360044A136070477C420050B8420050BA
:1013F000BC420050984200500023044A1360044A43
:101400001360044A1360044A136070471842005086
:10141000384200503C420050A04200500023044A91
:101420001360044A1360044A1360044A136070474F
:10143000A4420050A8420050AC4200506442005008
:101440000023044A1360044A1360044A1360044AE8
:101450001360704768420050884200508C42005030
:10146000FC4200500023044A1360044A1360044AFB
:101470001360044A13607047F8420050DC42005089
:10148000D84200504C42005070B5022809D00328C1
:1014900021D0002824D0164B00251E001900154C21
:1014A00004E00021124B0C001E00134D134A9481DE
:1014B00093805380D68011815581114A14788442DB
:1014C00007D000210F4B19700F4B8C420DD1022118
:1014D0001970107070BD0023074D1E001900DEE763
:1014E00003000100024E094DD9E70A28F0D1EEE7CA
:1014F0006D040000A604000032060000CC090020A4
:1015000088090020870900208609002019030000AF
:1015100070B5072200212D4807F0DAFDFF220023D5
:101520002B4D2C4E9200EA52F25202330E2BFAD17E
:10153000294C0120FFF788FE0020FFF7DFFEFA208C
:10154000013CC000A4B202F0EAFF002CF1D19134BA
:10155000FF340120013CFFF777FEA4B21F4802F0E0
:10156000DEFF002CF5D1FFF76BFFFFF77BFF1A4C76
:101570000020FFF701FD013C0020FFF757FDA4B25A
:10158000164802F0CCFF002CF2D1FFF711FFFFF755
:1015900021FF114C0020FFF7A3FD013C0020FFF7C5
:1015A000F9FDA4B20D4802F0BAFF002CF2D1FFF70A
:1015B00023FFFFF733FF0A20FFF766FF3100280003
:1015C0000E2207F04BFE200070BDC046E809002047
:1015D000DA090020CC09002035040000DC050000F9
:1015E000F0B5C04D85B02E78012E00D183E0022EDB
:1015F00000D11BE1002E00D042E1BB4EBB4C337842
:101600000193002B13D0013B3370B94B02931B782D
:101610000193002B33D0029A013B13702378DB43F4
:101620009B0700D080E02B7801332B707CE0B14F1A
:10163000B14B7A885B889A420CD90120FFF79CFC59
:10164000032333707B88013B01227B802378934303
:101650002370DAE79A4207D20198FFF78DFC032343
:1016600033707B880133EFE7FFF7A2FE0123227876
:1016700013432370019AA14B32701A80C5E79D4F26
:101680009D4BBA889B889E4E9A4215D90120FFF740
:10169000CDFCC8213388012249008B4200D204329C
:1016A000029901330A703380BB88013B0222BB8060
:1016B000237893432370B1E79A4210D20198FFF741
:1016C000B5FCC8213388012249008B4200D2043284
:1016D000029901330A703380BB880133E6E7FFF7D4
:1016E00079FE0223227813432370019B019A3380F1
:1016F000029B1A7092E7834B7C4C02931B780193F8
:10170000002B13D0029A013B13707F4B02931B787E
:101710000193002B4BD0029A013B13700C222378CB
:101720001340934200D17EE705B0F0BD714F724B7C
:10173000FA88DB88754903919A4217D93000FFF780
:10174000CFFCFF21039B32001B8849008B4200D84D
:101750000522029901330A70039A1380FB88013B2A
:101760000422FB80237893432370CEE79A4212D25F
:101770000198FFF7B5FCFF21039B32001B8849004D
:101780008B4200D80522029901330A70039A138014
:10179000FB880133E4E7FFF72FFE0423227813438D
:1017A0002370019A039B1A80029B1A70ADE7514F78
:1017B000514B3A891B89564903919A4216D9012007
:1017C000FFF7E8FCFF22039B52001B88934200D8DE
:1017D0000526029A01331670039A13803B89013B58
:1017E00008223B8123789343237097E79A4211D2D2
:1017F0000198FFF7CFFCFF22039B52001B88934206
:1018000000D80526029A01331670039A13803B898B
:101810000133E5E7FFF702FE082322781343237024
:10182000019A039B1A80029B1A7077E7394E2F4C5E
:1018300033780193002B02D0013B337011E02D4F20
:101840002D4B7A895B899A421CD90120FFF7FCFC59
:10185000032333707B89013B10227B8123789343E0
:1018600023702D4B02931B780193002B1CD0029AFE
:10187000013B1370302223781340934200D053E78A
:101880000023D2E69A4207D20198FFF7DDFC03233A
:1018900033707B890133DFE7FFF7D2FD1023227815
:1018A00013432370019BC8E7124F134BBA899B89DE
:1018B0001A4E9A4234D90120FFF720FDFF213388C8
:1018C000012249008B4200D80432029901330A7088
:1018D0003380BB89013B2022BB8123789343237053
:1018E000C8E7C046860900200600002087090020BE
:1018F00005000020DA090020CC090020840900201E
:10190000820900200400002003000020800900203C
:101910007E09002002000020010000207C09002038
:101920009A4210D20198FFF7E9FCFF213388012287
:1019300049008B4200D80432029901330A70338087
:10194000BB890133C7E7FFF78DFD202322781343BE
:101950002370019B019A3380029B1A708AE7C0466C
:10196000F8B5414B414A4248197812780478002969
:1019700003D140490978032960D100233E490B6017
:101980003E490B70FA213E4B3E4E5200955B0020C3
:10199000185E8900684304F0AFFC401905F0ACFD07
:1019A000FA21394B6400A45B051C0020185E8900F5
:1019B000604304F0A1FC001905F09EFD3349041CAE
:1019C000281C04F0ABFD00284AD10021281C04F09B
:1019D00091FD002800D000252C49201C04F09EFD1C
:1019E00000283FD10021201C04F084FD002800D0F5
:1019F0000024291C254805F015FB211C051C234843
:101A000005F010FB224F041C291C386804F06CFD03
:101A1000002804D1281C04F095FD02F0D9FE1D4ECB
:101A2000211C306804F060FD002804D1201C04F063
:101A300089FD02F0D9FE3D603460F8BD11001B78CD
:101A400021430B439ED10D490B780133DBB20B7060
:101A5000042B00D896E70120074B1860052390E778
:101A60000A4DB9E7094CC4E70111002063090020C1
:101A700062090020E40E00205C4200504D09002065
:101A8000F207002008000020F007002000401C465C
:101A9000540900205009002010B5274B1B78042B57
:101AA00023D0264B1B78002B1FD0254A254B1278BC
:101AB0001B789A4209D3244B1968244B002920D162
:101AC0001A78642A12D801321A70214A214B1278EE
:101AD0001B789A4209D3204B1968204B002922D148
:101AE0001A78642A15D801321A7010BD1970802333
:101AF0001B4A5B42117801200B431370FFF70AFA6F
:101B0000E3E700227F211A70154A13780B40137007
:101B1000DBE719702023124A012011780B43137060
:101B2000FFF7F8F9E1E7002220211A700C4A137838
:101B30008B431370D9E7C046031100200011002029
:101B4000630900207B090020A8080020A2080020CB
:101B5000620900206F090020A4080020A1080020CD
:101B60000008002010B5032841D82F4A2F4B013917
:101B700004F024FB1B17383E2D49097811702D4ABB
:101B8000127827E02C49097811702C4AF8E72C4983
:101B9000097811702B4AF3E72B49097811702B4A09
:101BA000EEE72B480478012C06D103291CD8080045
:101BB00004F0FAFAE2E8EDF200780328F5D1814268
:101BC00012D8080004F0FAFA02080A0C2149097830
:101BD000117000221A700AE01F49F8E71F49F6E762
:101BE0001F49F4E70329ECD900211170197010BDC9
:101BF0000329F9D8080004F0E1FA02070C11194989
:101C000009781170184ABBE7184909781170184A09
:101C1000B6E7184909781170174AB1E717490978EA
:101C20001170174AACE7C046610900206009002026
:101C30007B0900206F0900207A0900206E0900202E
:101C4000790900206D090020780900206C09002026
:101C50000211002077090020760900207509002074
:101C60007409002073090020670900207209002010
:101C70006609002071090020650900207009002014
:101C80006409002070B5334A334D1378002B02D11C
:101C900001212B7011700122304B28781A70062810
:101CA00055D82F4C04F08AFA040C212A37464B00F1
:101CB0000020FFF7E9FB322323802B78013312E069
:101CC0002388002B02D0013B23800DE0254A264BC0
:101CD00012781A70254A264B12781A70FA235B0084
:101CE0002380F33BFF3B2B7070BD2388002BEAD190
:101CF000204A214B12685A800323F4E71F4A1A4BEB
:101D000012781A701E4A1A4B12781A70C8235B0098
:101D100023808D3BE6E72388002BD4D11549164A52
:101D200009689180104A1370114A1370322323807E
:101D30002D3BD8E72388002BC5D10A20B9E723889B
:101D4000002BC0D101220F4B1A700723CBE70022D2
:101D50001A70C9E78C090020070000208D090020B7
:101D60008A0900207A090020610900206E090020FC
:101D700060090020A4080020C20900207909002081
:101D80006D090020EC0E002070B5314B31481978F8
:101D9000314B1A78314B8A420DD131490C78012CE4
:101DA00009D9002A07D0012202701A783B2A05D8E7
:101DB00001321A7070BD00220270FAE73C221A70DC
:101DC0000B78DCB2022B22D0032CF3D1254B9C885C
:101DD000254B186805F0D8FB244B051C988805F0A6
:101DE000D3FB011C281C05F01DF9051C200005F083
:101DF00083FB011C281C04F091FB0028DAD0002C86
:101E0000D8D002231A4A11780B431370D2E7154B2E
:101E10005D88154B186805F0B7FB144B061C5888F5
:101E200005F0B2FB011C301C05F0FCF8061C280074
:101E300005F062FB011C301C04F070FB0028B9D0D7
:101E4000002DB7D00A4B1A7814431C70B2E7C04675
:101E5000610900208F090020630900208E090020FD
:101E60000111002090090020A40800209A090020F8
:101E7000000800200022164B164970B518680C683F
:101E80000A601A6005F080FB134904F081FF061C0C
:101E9000200005F079FB104904F07AFF0F4904F0A7
:101EA00095FD0E49051C301C04F090FD0C49FEF711
:101EB00049FB04F047FB0B4C0B492060281CFEF744
:101EC00041FB04F03FFB094C2060FFF75DFF70BD54
:101ED000201100201C110020000070420000404131
:101EE000FC080020A8080020AC080020A40800205E
:101EF000354A70B513880500002B01D0013B1380D3
:101F0000324C2388002B25D1B42231482280067818
:101F1000304A042112789E4205D001399A4202D0FB
:101F2000B2425B4159182C4B027019702B4B1A7836
:101F30002B4B1A70284B1B78032B21D8012B37D839
:101F400020D02088002802D0013880B22080254B84
:101F50001D7070BDB42BEDD0782B20D11E4B1B789B
:101F6000013B032BEDD82048204AC3782049D37089
:101F7000CE78204BDE70007910710A791A71E0E793
:101F8000042BDED11848194A4378194953704E780A
:101F9000184B5E70807890708A789A70D1E73C2BED
:101FA000CFD10D4B1B78032B0BD8012BEAD8C8D10E
:101FB000114B1878114BC0B21978C9B2FFF7D2FD96
:101FC000BFE7042BBDD1F3E7EA1000209C080020F6
:101FD0009F080020A00800209B080020021100207C
:101FE0004C0900209E080020370F00203E0F0020E3
:101FF000290F0020300F00200311002001110020C4
:10200000F0B5994B994A85B0029303921B78984A90
:10201000984C994F994E9A4D0192002B34D12378C8
:10202000DAB20092002B2FD1964B1B78032B2BD0CA
:10203000039B5B78102B27D01000FEF76BFF009AF4
:10204000914B3A705A709A70DA701A715A719A718B
:10205000019B1A703378002B01D0013B33702B7831
:10206000002B01D0013B2B70FFF77AFC33782A78E4
:102070001343DBB2002B05D10A20FFF705FA0A2033
:10208000FFF736FF05B0F0BD039B5B78102B03D044
:102090007C4B1B78032B4AD1039B7C4A5B781370E3
:1020A0007B4B1B781A00103A102A2FD80023019A74
:1020B0000A2013703B70FFF7E7F9039B5B78102B46
:1020C0000FD0704B1B78032B0BD0724B1B88052B4A
:1020D00003D10023019A3B7013702078C0B2FFF740
:1020E00007FF019A33781278934200D8B1E0013BA0
:1020F00033702B783A78934200D8AFE0013B2B70D5
:10210000FFF72EFC2278644B1A70BBE70020042BEB
:1021100000D890E0052B01D103208CE0092B01D8D9
:10212000022088E0252BC8D1FFF7ACFDC5E70020D1
:102130005A4B22781870584B824218D11B78834230
:1021400003D1574B1B7883421BD10123544A137090
:102150004D4A53709370D370137153719371002370
:10216000019A3B70137005224A4B1A80A5E722782A
:10217000012A2AD11B789342E7D1494B1B78002BC7
:10218000E3D033782A781343DBB2002B03D0414BE2
:102190001B88052B91D00020FFF776F9414B1B7867
:1021A0003F2B8AD13B4B1B88012B06D1029B207809
:1021B0001978C0B2C9B2FFF7D5FC364A1388002B94
:1021C00000D17AE7013B138077E72278032A13D105
:1021D0001B789342B9D1324B1B78002BB5D03378A2
:1021E0002A781343DBB2002B04D02A4B1B88052B23
:1021F00000D162E70320CFE72278022A13D11B78AF
:102200009342A2D1264B1B78002B9ED033782A789C
:102210001343DBB2002B04D01E4B1B88052B00D1CF
:102220004BE70220B8E72378042B00D045E7184B92
:102230001B78042B09D8FFF727F91B4B019A1B7851
:1022400013701A4B1B783B7037E7052B00D067E7FC
:1022500062E7934200D34CE7013349E7934200D34E
:102260004EE701334BE7C046011100205909002019
:10227000610900200311002060090020630900208B
:1022800062090020E40E0020530F002058090020AE
:10229000F00E00205E090020000000208C090020C4
:1022A00000110020870900201A08002019080020CA
:1022B000AA2370B5174C184E23700023607098B293
:1022C0000025904200D2CD5CF5540133F02BF6D1BD
:1022D000F121124801F096FB2300020AF2331A7032
:1022E0002300F333187001230D4DF4222B602100DD
:1022F0000C4803F08BFE80220A4B92009969114230
:10230000FCD08022120199691142FCD000232B607D
:1023100070BDC046E50A0020E70A0020E60A00205A
:10232000584200500000154070B5204C0200207843
:10233000042839D803F042FF03070F1B1F000123B5
:10234000AA2A06D070BD1A4B1A700022194B1A70B7
:1023500002232370F6E7174815490378C91801339B
:10236000DBB24A700370EF2BECD90323F1E7124B79
:102370001A700423EDE7104B0D4D1E78F121360243
:102380002800164301F03EFBB0420DD10B4E3378CE
:10239000002B09D10A4B2A780A481A70691CF022CE
:1023A00006F05CFF012333700023D2E7AF0E00205C
:1023B000BC0D0020AE0E0020AD0E0020BB0D002095
:1023C000BA0D0020CA0C0020F0B50400EF22002155
:1023D00085B0013006F07CFEC24B1B782370012BC8
:1023E00000D07CE1C04A1278511E022900D8D318CF
:1023F0006370BE4BBE4F1B78BE4AA3703B78127809
:10240000E370BD4B511E8A411B78591E4842414121
:10241000043B500089000143584243410B43237160
:10242000B64B1B88591E8B41B5499B000978481E45
:10243000814149000B431A43B24B62711B78B24A87
:10244000A3715B0001929A5A110A2272AF4AE1719C
:102450009A5A110AA272AE4A61729A5A110AE1722C
:102460002273AC4AAC499B5A02911A0AA373AB4B34
:1024700062731B78012223742300A949A94D1133EB
:1024800003910299885C411E884103994000895C50
:102490004E1EB1410143A44819705100405A987032
:1024A000060AA2485E70405A060A1871A048DE70FB
:1024B000405E9871060A9F485E71415A080A197277
:1024C000D87168780121022801D80331091A59729C
:1024D00099490135895C0132997200212878D972B5
:1024E0001873387858730E33052ACAD1934B1A786B
:1024F000230049331A70924B1A7823004A3319701B
:102500005A70904B1A7823004C3319705A708E4BC6
:102510001A7823004E3319705A708C4B1A782300A6
:10252000503319705A708A4B1A782300523319703D
:102530005A70884B1A782300543319705A70864B9E
:102540001A782300563319705A70844B1A78230076
:10255000583319705A70824B1A7823005A33197005
:102560005A70804B1A7823005C3319705A707E4B76
:102570001A7823005E3319705A707C4B1A78230046
:10258000603319705A707A4B1A78230062331970CD
:102590005A70784B1A782300643319705A70764B4E
:1025A0001A782300663319705A70744B1A78230016
:1025B000683319705A70724B544F1A7823006A337B
:1025C00019705A706F4B524D1A78230051486C3372
:1025D00019705A700233019A525A160A1E705A70B4
:1025E0007A5A160A9E70DA706A5A160A1E715A7161
:1025F000425A0231160A9E71DA7108330629EAD16D
:10260000220000236049614D019161499E3202918F
:1026100060490391019E1000B446002118389C4483
:102620006646765A0231370A07704670023008292A
:10263000F6D1029E1000B446002110389C44664634
:10264000765A0231370A0770467002300829F6D1EF
:10265000039E1000B446002108389C446646765A12
:102660000231370A0770467002300829F6D15E1928
:1026700010000021B4466646765A0231370A0770C8
:10268000467002300829F6D15B182032182BC1D1D0
:10269000230027004049414AE633EE3700200E5E12
:1026A0000020155E0020864203DBFF30864200DCFE
:1026B000300018700020854203DBFF30854200DCCB
:1026C000280058700233023102329F42E6D1344B67
:1026D000EF341B881A0A3A70237005B0F0BD00234E
:1026E00086E6C0460011002003110020D210002011
:1026F00001110020DF100020060F0020061100202D
:10270000B60E0020D6000020E4000020DE000020ED
:10271000D8000020EA000020300F00200008002030
:102720003E0F0020D6100020BE0F0020A20F002078
:10273000780F00205C0F0020080F0020C90C00203B
:102740007B0900206F0900207A0900206E09002013
:10275000790900206D090020780900206C0900200B
:102760007309002067090020770900206B09002009
:10277000760900206A0900207509002069090020F7
:10278000740900206809002038010020F0000020B2
:102790002001002008010020880F0020960F002053
:1027A000120F002070B5B84EBEB03378002B00D1A8
:1027B000C2E0B64B02ACF0222000B5491D7806F00D
:1027C0004DFD0023681E33700D2800D9A2E003F0F0
:1027D000FFFC0E003D0072008700BD00C300C90071
:1027E000F3000C014B0016011801B901DC0122783D
:1027F000A8481300591E8B41A749A84C0B70A84943
:102800004B708B70CB700B714B718B71A549A64BC4
:10281000002A16D1227002700A701A700023A34A8F
:10282000A34953709370D3701371A24A4B708B708D
:10283000CB700B71117843330B4313709E4B012205
:1028400088E00022227002700132E5E72078924B86
:1028500000280BD1187000210022944B5A709A70F6
:10286000DA701A71914255D1002354E001220138E7
:1028700011001A700328EFD8864B03F09FFC020367
:10288000181A00221A701A7884490A7001210C0063
:10289000884A1B781078044314708B42DBD0814B3C
:1028A0001970814B1970032303431370D3E702227D
:1028B000E8E70322E6E723787B497A4A13700B7036
:1028C00002237C49087803430B70744B1978012963
:1028D000CAD018781178C0B2C9B2FFF743F9C3E77C
:1028E0002378012B0CD16378744A591E8B419B00CD
:1028F000137000226D4B5A709A70DA701A71B3E738
:10290000022B05D162786E4B511E8A411A70F0E796
:10291000032B13D0012301A9022282200D704B70DA
:10292000FFF7C6FC0A2D07D16648FFF74DFDF022E0
:1029300081206449FFF7BCFC3EB070BD62785F4BFC
:10294000511E8A411A7002225F4BDFE75C4B2278EE
:10295000511E8A411A7087E723785C4A022BD9D826
:10296000137027E02378022BD4D809226A44107808
:1029700052785749120202435B0052BA5A520B2254
:102980006A441078527853491202024352BA5A529A
:102990000D226A44107852784F491202024352BA0B
:1029A0005A520F226A44107852784C49120202435C
:1029B00052BA5A524A4B42E723785A1E032AA9D8E0
:1029C000A278002A00D06E226178002907D14549FB
:1029D000CA544549CA54354A0121D15444E7012912
:1029E00098D14249CA544249F4E723785A1E032A2F
:1029F00000D98FE73F4A6178D1542D4AECE73E4B2E
:102A0000A5E721786078E2786379002917D1013849
:102A1000032800D97EE703F0D1FB02060A0E3749EE
:102A20000A70374A9CE737490A70374A98E73749AE
:102A30000A70374A94E737490A70374A90E7012904
:102A400006D1884200D065E734490A70344A87E7E6
:102A5000022900D05EE70138032800D95AE703F0C5
:102A6000ADFB02060A0E2F490A702F4A78E72F495C
:102A70000A702F4A74E72F490A702F4A70E72F49CE
:102A80000A702F4A6CE7C046BB0D0020BA0D00202B
:102A9000CA0C0020F30E00200011002003110020BA
:102AA000530F002001110020F20E00201B0F002008
:102AB000140F0020EB0E0020EA0E0020060F00206D
:102AC000DF100020D90B0020050F0020D6000020C9
:102AD000E4000020DE000020D8000020EA000020F2
:102AE000EC0E00203E0F0020370F0020300F00209A
:102AF000290F0020080F0020C90C00207B090020AE
:102B00006F0900207A0900206E0900207909002051
:102B10006D090020780900206C090020730900204D
:102B200067090020770900206B0900207609002042
:102B30006A09002075090020690900207409002035
:102B4000680900202378022B00D9E3E66278032A83
:102B500000D9DFE6DB00002A0DD1114A9B181800CE
:102B60000830A178E27809020A431A80023302345D
:102B70008342F6D11EE7012A01D10A4AEEE7022A72
:102B800001D1094AEAE7094AE8E72178082900D98A
:102B9000C0E6E12212014A43054B1A8064E6C046B2
:102BA000380100202001002008010020F000002052
:102BB000120F002010B50448FFF706FCF022812018
:102BC0000149FFF775FB10BDF5090020044B10B556
:102BD0001A69D20703D51868C0B2FFF7A5FB10BD6C
:102BE0000000154010B5FFF7F1FF10BD03004118BC
:102BF00000208B4200D170471A7801335040C0B298
:102C0000F7E7000070B5194B05001B78184C002B36
:102C100000D123702078082825D803F0CFFA050CBE
:102C20001515151515151A00AA2D03D101232370AA
:102C3000104B1D7070BD2B00113B5A4253415A1C62
:102C400022700C4AD554F5E7431C2370094B1D54E0
:102C5000F0E7084808210572FFF7C8FFA84202D133
:102C60000122054B1A7000232370E3E708110020AE
:102C7000B50E0020BC0E0020B70E0020064B10B58C
:102C80001A69D20706D51868C0B2FFF7BBFF0A223F
:102C9000024B1A7010BDC04600000540081100200C
:102CA00010B5FFF7EBFF10BDAA2370B5164C012637
:102CB0002370893B6370154B08211B782000E3705B
:102CC000134BA6701B78134D2371134B1B78637144
:102CD000124B1B78A3710023E371FFF787FF0922D2
:102CE000207221000E482E6003F090F980220C4BD8
:102CF000920099691142FCD0802212019969114217
:102D0000FCD000232B6070BDD00E002003110020EA
:102D10000111002048420050DF100020BB0E0020AF
:102D20000000054010B50C4B1A78012A09D1002289
:102D30001A700A4B0A4A1A800A4A0B4BD2781A7048
:102D400010BD0A4B1A88002AFAD1F532FF321A80D8
:102D5000FFF7AAFFF4E7C046B70E002006110020D7
:102D6000DC050000BC0E0020B60E00200A11002079
:102D7000F7B54A490878002874D0494B00201B78E1
:102D8000012B6FD0474A484E10783378474C019258
:102D9000834253D0464A00282DD183422DD0454F3F
:102DA00045493878087039784448CDB2012902D1B4
:102DB0000178002901D001780D0041490D700021F2
:102DC0003970404F3970191C042B00D9042101704F
:102DD00011703D4A3D4B1168002905D0002010605C
:102DE000042219780A431A70032219780A431A70C8
:102DF0001E23237022E0002B35D12F4B2D481B784A
:102E00000370304803702E4B2C481B7803701370EE
:102E10002D4A2E4B1068002805D000271760042289
:102E2000187802431A704322187802431A7000235C
:102E3000274A23701370274A0B7013802378002BC6
:102E40000CD0013BDBB22370002B07D10122204BB9
:102E50001A7040231D4A11780B43137001203378F8
:102E6000019A1370FEBD191C042B00D9042110789F
:102E7000CBB29842E2D00223104F39701170134A3E
:102E800011780B4313700B4B1A78012AB0D01878C5
:102E90003978C0B2C9B2FEF765FEA9E7DF1000209D
:102EA000B40E0020B10E0020B60E0020B00E00209F
:102EB000F20E002003110020E1100020011100207B
:102EC000E0100020F30E0020F40E0020EB0E002096
:102ED000E50E0020B20E002030B51C4B0200197820
:102EE0001B4B002900D1197018780E282CD803F03C
:102EF00065F9080F0F0F0F0F0F0F0F0F0F0F0F14A4
:102F00002300AA2A08D101211970124B1A7003E07C
:102F1000411C19700F4B1A5430BD002001000D4C9C
:102F2000255C01306940C9B20D28F9D18A420BD124
:102F30000E2162731970EFE7EE2A05D13221064A9D
:102F40001180064A313911700022DFE7FC0E0020A3
:102F5000FB0E0020DC0F002010110020B410002018
:102F60000B490C4B0A78002A04D11A700A4B1A70CC
:102F70000A4B03E01A78092A02D801321A70704706
:102F80000A221A7000220A700121034B1970EFE720
:102F9000FA0E0020F90E0020F80E0020E40E0020AA
:102FA000AA22244B1A7000225A70234A11781278F0
:102FB00099702249012A02D1214A12780A700A78AE
:102FC0002049DA70204A0978127820481A71204A7C
:102FD000007812780A431F49097809010A43002141
:102FE0005A711D4A997112780243DA711B4A1268AC
:102FF0008A4204DA013119721432110003E01972A5
:10300000FF21642AF8D1164A59721168FF226429F7
:1030100001D00A0014329A7200221100DA721A7377
:10302000985C013241400D2AFAD1E13259739A730A
:103030007047C0461D100020031100200111002020
:10304000F20E0020E80E002002110020E90E002000
:10305000E70E0020E60E002000080020F807002000
:10306000F4070020AA220F4B01211A702A3A5A7045
:1030700000220420997019721100187101385871DA
:103080001330DA709871DA715A729A72DA721A73AE
:10309000985C013241400D2AFAD1E13259739A739A
:1030A0007047C0461D100020AA22114B1A70293A01
:1030B0005A70403A9A700F4A1268110AD970422128
:1030C0001A71002299710C495A7109685A72080ADA
:1030D00019721100D8719A72DA721A73985C0132FF
:1030E00041400D2AFAD1E13259739A737047C046B4
:1030F0001D100020A8080020A4080020AA22144BBC
:1031000014491A70A53A5A70043A9A700A881248FB
:10311000120ADA700A880221997101881A71090A63
:10312000D97101880022197203210C489972018813
:103130005A71090AD97201885A7219731100985C80
:10314000013241400D2AFAD1E13259739A73704726
:103150001D100020F8100020F6100020F4100020B0
:10316000AA22194B1A70A03A5A70184A11780129EC
:1031700023D100229A700A00DA70154A12781A7167
:1031800000225A718032012905D1124A1278013A7F
:1031900051424A4180329A7100221100DA711A724A
:1031A0005A729A72DA721A73985C013241400D2A8F
:1031B000FAD1E13259739A737047074A12789A70BC
:1031C000064A1278D8E7C0461D100020E50E002000
:1031D00002110020DF100020F30E0020F20E00206C
:1031E000F7B5C24BC24A5E781670122E15D8300061
:1031F00002F0EEFF1D009F00EA014902A702CA0289
:10320000C502D3021C001C006D031C001C001C0026
:103210001C001C001C001C002402802E00D130E386
:10322000812E00D130E3222E00D14AE3F7BD57248E
:10323000B04A1178A1431170D87911782040014328
:103240001170AD4AAD4915780092072209782A40DD
:103250000A43D2B2AA4C002A59D0AA4A1378012BA9
:103260000AD1A94B1B78002B06D1A84913700B80FB
:1032700040331D43009B1D70AA232370A33B637042
:10328000A34BA44A1B781278A370A34B28001B7889
:10329000E370A24B1B782371A14B1B781343A14A07
:1032A00012781201134363710023A371E371237237
:1032B0006372043318401D4226D0E1219A4F033B2C
:1032C0003868A372090102F08DFFE121E072090163
:1032D000386803F00DF808003C2102F083FF00235A
:1032E0002073E25C013356400D2BFAD1E133A37316
:1032F0006F3B009AFF3B2B43667313700F22210034
:103300008A4802F09FFD91E7A072E072E7E76D0640
:1033100002D5FFF725FFF1E7E122D97A12014A43EE
:10332000197B3C234B43D3187F4A1360FFF738FEC9
:10333000E4E77F4A9D787F4815701178012901D014
:10334000D97801700178002904D05F26694C217872
:10335000314021706849694E0C78A44600240C570E
:10336000002C5CDA002415700C701178347001297F
:1033700001D0D9780170597901250E006E4C2E408C
:10338000267010266D4C31402170D9796C4C294043
:10339000257829432170997A012909D1E121DC7A24
:1033A000090161431C7B3C236343CB185E490B60DE
:1033B0001378002B00D086E00121624B5970997080
:1033C000D97019715971997101235F490478CC54EE
:1033D0000133072BFAD14A49A3330B7013784D4AB6
:1033E0008B7003781278CB704D4B01241B785748B3
:1033F00013434C4A007812784C7012011343002298
:103400004B713C4B8A711B780343CB71504B1B684B
:10341000934200DBBCE00C7214331A00BDE00324BD
:10342000674636783C403443E4B2002CA3D1384C94
:10343000157000942570DC78374D04702C7004787A
:10344000002C34D11478002C31D1424C424E2478D7
:103450003578A54210D0414D2D78012D0CD1270093
:103460003F4D347001957D1EAF41019D2F70802727
:103470003C4D2C703C4D2F7000243C4D66462C700A
:10348000009D2C703A4D2C70234D2C700325354334
:103490000D70384D384E2C70384D36782C70384DB4
:1034A0002C80384D2C70384D2E70384D2C70154CAA
:1034B0002578012D00D05EE70025257040240D7889
:1034C0002C430C7057E71378012B02D102211D4BBE
:1034D00074E71378032B02D104211A4B6EE713789B
:1034E000022B00D070E70821164B67E7DC0F0020A5
:1034F000E40E002000080020EB0E0020EA0E002061
:103500001D100020E50E0020B00E0020B20E00209D
:10351000F30E0020E80E0020F20E00200211002021
:10352000E70E0020E60E0020F40E002000001940F7
:103530000311002001110020EF0E0020EE0E0020EC
:10354000ED0E00204C0F0020450F0020E90E00205A
:10355000F8070020E2100020B60E0020DF10002047
:10356000BA0E0020B90E0020B80E0020E110002095
:10357000E0100020FD0E0020050F0020060F0020A7
:10358000E4100020E6100020040F0020B40E0020FC
:103590000A72FF22642B00D03EE7CF4B4A721A68B2
:1035A000FF23642A01D0130014338B7200231A0006
:1035B000CB720B73C85C013342400D2BFAD1E1335F
:1035C0004A738B730F229BE60022C4490A70C449D8
:1035D0000A70C4490A70C4490A60C4490A709B78D9
:1035E000C3490B70AA23C3490B70A83B4B700E3321
:1035F0000B71C14B8A701B78CA704B71BF4B1B7823
:103600008B71BF4B1B78CB71BE4B1B780B72BE4BC3
:103610001B784B72BD4B1B788B72BD4B1B78CB72EA
:10362000BC4B1B780B731300885C013243400D2A9E
:10363000FAD14B73EE2302328B7361E6AA23102278
:10364000AC490B70983B4B7000230A71B24A8B70E7
:103650001278CB704A71B14ACB7212780B738A71AF
:10366000AF4A1278CA71AF4A12780A72AE4A12781B
:103670004A72AE4A12788A721A00C85C013342401C
:103680000D2BFAD19BE7DD78A94A681E15705C798D
:103690001A7908280BD8002302F090FD0530343841
:1036A0003C4045494D00A34B1A70A34B1C70AB1F07
:1036B0000021032B00D92100A04B1A70A04B1970D8
:1036C000AA238C490B70A73B4B7000230A719D4ABB
:1036D0008B701268CD70100A8A729B4A4872126809
:1036E0004C71100A0A731A008B71CB710B72C8727D
:1036F000C85C013342400D2BFAD160E7934B1A703E
:10370000934BD3E7934B1A70934BCFE7934B1A70BD
:10371000934BCBE7934B1A70934BC7E793490A70CF
:1037200093490B70C3E793490A709349F9E79349AA
:103730000A7093490B700021924B1A70924B1970CA
:10374000B5E79A78654B6B491A7001228F4B1A7056
:10375000AA230B70A63B4B7000231A008B70CB7012
:103760000B714B718B71CB710B724B728B72CB7275
:103770000B73C85C013342400D2BFAD11FE72021A7
:10378000834A13788B43A0E01021814A13788B433E
:103790001370FFF7B3FC574914E700277C4C7D4EAC
:1037A000E75722787C487D494C4D002F44DA7F272B
:1037B0003A402270002232709A782A702A78012AC0
:1037C00002D0DD78464A15705A7901251700744EEB
:1037D0002F4037701027734E3A403270724ADE79AC
:1037E00017783E431670E122DE7A120172431E7B87
:1037F0003C237343D3183C4A1360384B00781B7842
:10380000984202D12378AB432370354B09781B785B
:10381000994203D1022123788B4323701168634BB3
:1038200000291BD11B688B4203D1042223789343C8
:103830002370FFF7B5FBAEE7032736783A403243F3
:10384000D2B2002AC0D19A782A7002702A78012A4E
:10385000BAD0DA78224D2A700A70B5E719680029C3
:10386000E7D0E1211068090101381D6802F0BAFCB7
:10387000E12106000901681E02F0B4FC8642D8D19D
:10388000D3E7FFF7EFFB86E74948997802780129EB
:1038900014D10A4302241100DD78A143012D01D186
:1038A0002100114304221C790B009343012C01D108
:1038B00013000B430370FFF7F7FB6CE701218A430A
:1038C000E8E75F21094A13780B401370B1E7304AEB
:1038D0004021137856E7C046F4070020031100206A
:1038E00001110020DB0F0020FC1000200008002048
:1038F000F10E00201D1000207B0900206F09002020
:103900007A0900206E090020790900206D09002045
:10391000780900206C090020730900206709002045
:10392000770900207609002075090020740900201D
:10393000F00E0020180800200C0800201A080020B3
:1039400019080020A8080020A4080020170800205B
:103950000B080020160800200A0800201508002087
:103960000908002010080020040800201408002086
:103970000808002013080020070800201208002073
:10398000060800201108002005080020EC0E002089
:10399000EB0E0020EA0E0020F30E0020F20E0020B5
:1039A000EF0E0020EE0E0020ED0E0020F40E0020A1
:1039B000E90E002070B5084B1A78D5B2012A0AD159
:1039C000064A1488002C06D11C70FFF709FC044B32
:1039D0001D70044B1C7070BDB4100020101100202D
:1039E000FA0E0020F90E0020044B10B51868C0B282
:1039F000FFF772FA3222024B1A7010BD0000194014
:103A0000FC0E0020FF22130070B5094D094E00295D
:103A100003D11802104380B270BD047801395C40B4
:103A2000E4B22B5D89B253400130325DEFE7C0460E
:103A3000E4A90000E4A8000070B5384A0300127839
:103A4000374D002A00D12A702A78042A06D8501E41
:103A5000032812D802F0B2FB181F2A32252A07D8F1
:103A600030481C2A00D835D0511C2970835411E0ED
:103A7000262A43D000232B700CE0AA2B0AD1012266
:103A80002A70284A137005E0012B03D102222A7004
:103A9000244A537070BD03222A70224A9370224A2E
:103AA000032B01D1013BEDE70123EBE704222A7050
:103AB0001C4AD37027221D4B1A70EBE705222A708F
:103AC000184A1371184A1278022AE3D1013B934233
:103AD000E0D8EFE71D222A70144A037712781D2AD6
:103AE000D8D11B21C47E24021C19A4B2FFF78AFF7F
:103AF000A042BFD101220E4B1A70BBE727222A70C9
:103B00000C4A0848D377094A1278272AC2D1821D65
:103B1000D27F252112029B189CB2E7E7FC0E002001
:103B20000F0F0020F50F0020100F00200E0F0020B7
:103B3000B5100020FC0F0020F8B5AA23AB4CAC4D0B
:103B400023709A3B6370AB4B1B78A370012B4CD155
:103B5000A94B1A78A949AA4F895C00236171B95C05
:103B6000E270A171A7492371895CE171A6497F7850
:103B70008E5CA6492672885CA5496072895C8C4679
:103B80006046A449A072895CA34AE172022F00D06A
:103B900087E2A2490968080A6173A149207309688C
:103BA000080AA073E173117823746374A374E37437
:103BB00023756375A375E3752376637613781B21EC
:103BC0002000A376FFF71EFF030AE3760123207788
:103BD0001D222B602100934802F034F980239B00C2
:103BE000904A126A1A42FBD0C0E1022B01D18E4BDF
:103BF000AFE700210A00032BACD18C4A11708C492D
:103C00000878012863D1013B0B700523894FE370CD
:103C10003E78012E67D1884B884A1B7812786371F1
:103C2000874BE2731B78874AA371874B12781B7806
:103C30002671E371854B1B211B7820002372844B76
:103C40001B786372834B1B78A372834B1B78E372E0
:103C5000824B1B78237300236373A3732274804AFF
:103C600063751278A37562747E4AE37512782376C1
:103C7000A2747D4A63761278A376E2747B4A127846
:103C80002275FFF7BFFE030AE37620771D2221008D
:103C900064482E6002F0D6F880239B00614A126AC5
:103CA0001A42FBD0C82000F03AFC00232B603B7086
:103CB000504B1978012900D0F8E14F4A1078441888
:103CC0001470032802D9022018701170F8BD022860
:103CD00003D10B701123137097E7032895D10123AB
:103CE0000B701133F7E7022E3CD1614B614A1B7810
:103CF00012786371604B62741B78604AA371604BE9
:103D000012781B781B21E3715E4B20001B78A27494
:103D100023725D4B26711B7863725C4B1B78A37218
:103D20000023E37223736373A373E3732374E37455
:103D300023756375A375E37523766376A376FFF722
:103D400061FE030AE376012320771D222B60210008
:103D5000344802F077F880239B00324A126A1A42F4
:103D6000FBD09FE7032E00D09AE0494926714B888B
:103D7000484A63711B0AA37153882000E3711B0A30
:103D800023728B88444963721B0AA3729388434A47
:103D9000E3721B0A23734B8863731B0AA373538854
:103DA000E3731B0A23748B881B2163741B0AA3749F
:103DB0009388E3741B0A237500236375A375E37569
:103DC00023766376A376FFF71DFE030AE3760123CD
:103DD00020771D222B602100124802F033F8802347
:103DE0009B00104A126A1A42FBD05BE73610002093
:103DF0009C420050D0000020D3000020530F002030
:103E00004C0F0020450F0020080F0020220F00203B
:103E10003E0F0020300F002000080020A8080020DE
:103E2000A408002000001B40D2000020070F002043
:103E3000D10000205A0F00207B09002077090020C4
:103E40006F0900206B0900207A0900206E0900200C
:103E5000790900206D090020780900206C090020F4
:103E6000760900206A0900207509002069090020F0
:103E700073090020D500002067090020D40000202D
:103E800072090020660900207109002065090020E0
:103E9000C2090020B8090020AE090020A4090020B2
:103EA00013788C4A9446112B66D12371D3888A48A3
:103EB0001A0A6271A3710622835E88491A12E2719E
:103EC000237206228B5E1A126272854AA372D3880D
:103ED00023731E0A834BE6720627DE5FA673371232
:103EE0000026E67326746674A674E67426756675F5
:103EF000664667733689370AE675A7750826805FB8
:103F00000612267660760820095E0812E176A07611
:103F10001289110A2177627708229B5E1A12E377D1
:103F20000023A277621CD3776F4AA11C1378002369
:103F3000CB771178E21CD177221DD3772521621D22
:103F40002000D377FFF75EFDA31D020ADA77E31D99
:103F5000D877012327222B602100644801F072FFEB
:103F600080239B00614A126A1A42FBD0C82000F0ED
:103F7000D6FA00232B609BE6122B39D1237153898B
:103F800055481A0A6271A3710A22835E53491A12B4
:103F9000E27123720A228B5E1A126272504AA37275
:103FA000538923731E0A4F4BE6720A27DE5FA673FE
:103FB00037120026E67326746674A674E6742675B6
:103FC000667566466773B689370AE675A7750C2667
:103FD000805F0612267660760C20095E0812E17674
:103FE000A0769289110A217762770C229B5E95E771
:103FF000002323713E4B3F4F5E783F4B66715878EC
:104000003E4BA07159783B78E1715A0603D5802266
:10401000524232436271DA0703D580225242024390
:10402000A2719B0703D580235B420B43E3710023FE
:10403000334A3B70127823726272324AA372E3727F
:1040400023735288A273110A6246617352882274E4
:10405000110A214AE1730221525E1112A2741F4A11
:1040600061740221525E111222751D4AE174528858
:10407000E375110A23766376A3761A4BA2756175F0
:1040800002229B5E1A12E2761F4A237713881B0ACC
:10409000637713881D4AA37713881B0AE377138875
:1040A00040E723736373A373E3737CE5184A022923
:1040B00009D11178032901D8013106E601211170D7
:1040C00003221A7002E60121124811700170197062
:1040D000FCE5C046A20F0020940F0020860F0020B0
:1040E0005C0F0020780F00200008002000001B401B
:1040F000530F0020EB0E00204C0F0020450F002036
:10410000EE0E0020BE0F0020F6100020F41000205C
:10411000D2000020D300002010B525488378022B60
:1041200040D1427B047BC3781202224922435B00C8
:1041300052BA5A52C27B847B12021F49224352BA9E
:104140005A52427C047C12021C49224352BA5A52EF
:10415000C27C847C12021A49224352BA5A52427DCE
:10416000047D12021749224352BA5A52C27D847DFD
:1041700012021549224352BA5A52427E047E12025A
:104180001249224352BA5A52C27E847E1202104908
:10419000224352BA5A52427F047F12020D492243EF
:1041A00052BA5A522822002104F092FF10BDC04694
:1041B000F50F0020A20F0020B00F0020BE0F00203E
:1041C000CC0F0020940F0020860F0020780F0020D5
:1041D0006A0F00205C0F002010B5824B82481979CD
:1041E000DA780170102900D06DE05A79022A36D0B1
:1041F000032A4FD0012A2BD199797C4A7C4811702F
:10420000D9797C4A1170197A7B4A1170597A7B4AA4
:104210001170997A7A4A1170D97A7A4A1170DA7CD7
:10422000997C12020A4352BA774942805A7D1C7D1A
:104230001202224352BA4A80DA7D9C7D1202224346
:1042400052BA82805A7E187E1202024352BA8A8083
:10425000997F6E4A1170DB7F6D4A137010BD99799A
:104260006C4A6D481170D9796C4A1170197A6C4A90
:104270001170597A6B4A1170997A6B4A1170D97A18
:104280006A4A1170DA7C997C12020A4352BA684970
:104290004280CBE79979674A1170D979664A1170E3
:1042A000197A664A1170597A654A1170997A654A85
:1042B0001170D97A644A11705A1DD27F012AC7D170
:1042C00062490A70C4E70029C8D1052A69D10520CE
:1042D00018565A795E49002805DA7F2002405D4869
:1042E0004A708A71027006229A569879002A14DA66
:1042F0007F221040584A50709070D07010715071E9
:1043000090710138554A072847D801F057FF4604F5
:104310004642464646440120107007229A56DC79F0
:10432000002A0ADA7F224E48224042708270C27010
:104330000271427182714B4802701A7A7F2A06D943
:104340007F221440E12212016243474802600922A1
:104350009A56587A002A03DA0124444A2040107001
:104360009A7A012A03D14248047822430270DB7D05
:1043700001201A0002408A709A07D20FCA705A07A9
:10438000D20F1C000A7108221440134207D0487152
:1043900064E70320C0E70220BEE70020BCE74C71C1
:1043A0005CE7002A00D159E70521595658790029C0
:1043B00003DA7F24264920408854062159569879EB
:1043C000002903DA7F24244920408854D979DB79F5
:1043D0005BB2002B00DB41E77F20214B0140995469
:1043E0003CE7C046F50F00205A0F00207B09002053
:1043F000C20900206F0900207A0900206E09002000
:10440000790900206D090020B8090020D50000209E
:10441000D400002077090020AE0900206B0900209D
:10442000760900206A09002075090020690900202A
:10443000A4090020730900206709002072090020E8
:10444000660900207109002065090020EC0E00209B
:10445000530F0020001100204C0F002003110020FA
:10446000450F002001110020F40E0020EF0E002067
:10447000ED0E0020044B10B51868C0B2FFF7DCFA4F
:104480003222024B1A7010BD00001B40FC0E0020AF
:1044900010B50D4B1A78012A0DD100221A700B4B62
:1044A0001B78012B02D1FFF737FE10BD022BFCD188
:1044B000FFF792FEF9E7064B1A88002AF5D164321D
:1044C0001A80FFF739FBF0E7B5100020100F00202D
:1044D0000C110020F0B50E880024B51AADB285424B
:1044E0001BD24F88864204D2BD1AADB20134854238
:1044F00013D28E88874204D2B51AADB20224854207
:104500000BD2C988B04204D98A1A92B203249042CD
:1045100003D90424884200D81C002000F0BD10B547
:1045200001F0DCFA10BD10B50400002C00D110BD64
:10453000FA208000013C01F0D1FAF6E710B50848F6
:1045400001F0A8FCE1210748490201F01FFD01210B
:10455000044801F016FD8022034B52011A6010BD81
:10456000100000040000054000E100E010B508481C
:1045700001F090FCE1210748490201F007FD01210B
:10458000044801F0FEFC8022034B92011A6010BD2A
:10459000110000040000154000E100E0962110B574
:1045A000064CC900200001F033FC0123A26913432B
:1045B0008022A361024B92031A6010BD00001940D3
:1045C00000E100E0E12110B5064C4902200001F0B5
:1045D0001FFC0123A26913438022A361024BD20373
:1045E0001A6010BD00001B4000E100E080220B4B70
:1045F0009201196A114208D01A620122084B1A630B
:10460000084A13680133136070471A6A1A62064B2E
:104610001A6A1A62054B1A6A1A62F5E700400050DE
:10462000000200501C11002040400050804000500B
:1046300020220B4B196A114208D01A62094B1F3A0B
:104640001A63094A1368013313607047074A116AF5
:1046500011621A6A1A62064B1A6A1A62F5E7C046B4
:10466000004100500002005020110020C0400050C6
:10467000404100502B4A1378002B01D0013B1370AE
:10468000294A1388002B01D0013B1380274A138845
:10469000002B01D0013B1380254A1388002B01D049
:1046A000013B1380234A1378002B01D0013B137088
:1046B000214A1378002B01D0013B13701F4A137855
:1046C000002B01D0013B13701D4A1388002B01D031
:1046D000013B13801B4B1A88002A02D01A88013A2A
:1046E0001A80194B1A88002A02D01A88013A1A80B7
:1046F000164B1A88002A02D01A88013A1A80144BE5
:104700001A88002A02D01A88013A1A80114B1A8896
:10471000002A02D01A88013A1A8001220E4B1A612F
:104720007047C046081100200A1100200611002021
:104730000C1100200E1100200F110020FC0E002093
:104740001011002018110020161100201411002053
:10475000520100201211002000000140FA2210B581
:10476000084C10212000920001F0E2FB012380217F
:10477000E26849001A43E260034A11602268134369
:10478000236010BD0000014000E100E010B5FCF71F
:1047900027FF0122014B1A6110BDC04600010140F4
:1047A000FA2210B5084C10212000920001F0C0FB45
:1047B00001238021E26889001A43E260034A116004
:1047C00022681343236010BD0001014000E100E0B6
:1047D000FA2210B5030000210248920000F018FFF1
:1047E00010BDC04600001440FA2210B5030000219D
:1047F0000248920000F00CFF10BDC04600000440CB
:10480000FA2210B500210E4B92000E4800F000FF76
:10481000FA220B4B920000210B4800F0F9FE012117
:10482000084800F0C6FF0121074800F0C2FF01213F
:10483000044800F0A9FF0121034800F0A5FF10BDC6
:10484000102700000000044000001440074A012324
:10485000916D08001840194201D005490B700721DD
:10486000936D8B43034393657047C04600000E4031
:104870000411002010B5124C1F2308220021200033
:1048800001F0A2F8A36C0F4A802113400122A36417
:10489000A36C49021343A364A36D0B42FCD0636E67
:1048A0001342F9D00121064801F0A6F88022064BF8
:1048B00092051A608023A26C1B011343A36410BDF0
:1048C00000000E40FFFFFCFF00E100E0F8B580258E
:1048D0003D4CAD0129002000002201F0FFF9636A80
:1048E00020001D43656201220D2101F00BFA802199
:1048F00020260025354F20000022090101F0EEF9A5
:1049000038000022202101F0E9F97B6A38003343A6
:104910007B620122052101F0F5F9012280212C485A
:1049200001F0DCF92B4B01221D6040212A4801F0E7
:10493000D5F92A4B01221D600421274801F0CEF948
:10494000274B01221D608021234801F0C7F9254B28
:1049500001352A001D603100200001F0BFF98021DF
:10496000214B2A001D602000C90001F0B7F91F4B40
:104970002A001D6004211E4801F0B0F900221D4BE1
:1049800020001A601C492A0001F0A8F92A001B49DE
:10499000114801F0A3F92A0019490D4801F09EF9C8
:1049A0002A001849184801F099F91022174B1A608B
:1049B0001E60174B1E60802362695B0113436361B5
:1049C0007B691E437E61F8BD0040005000410050ED
:1049D000804000509C4200504040005058420050DF
:1049E000484200505C42005014420050284200509F
:1049F000404100504843005040C0000008F700000C
:104A00004CCF0000C0C00000C040005000E100E0FA
:104A10008041005070B5A024592216218820E40559
:104A2000434D6B68012B00D07DE00C2001F0BAF8FB
:104A3000182001F081F80021072001F08FF8C02034
:104A4000C00501F03DF83B4801F03AF83A4801F062
:104A500037F83A4801F034F8394801F031F839486C
:104A600001F02EF8384801F02BF8384801F028F80A
:104A7000374801F025F8374801F022F8364801F0B0
:104A80001FF8364801F01CF8354801F019F8E0200D
:104A9000000601F015F800220C21264800F0E6FF80
:104AA00000223021244800F0E1FF00223021234879
:104AB00000F0DCFFA02280212248D205090300F08B
:104AC000D5FF802100222048090300F0CFFF80217C
:104AD00000222048C90000F0C9FF802100221E48A2
:104AE000C90100F0C3FF002203211C4800F0BEFFF3
:104AF000002203211A4800F0B9FF01F0F1FA194B26
:104B000044226363184B236380235B01E363174BE9
:104B1000A3630023636422643332E364A3642365E4
:104B2000A2656B6070BD6A606960686078E7C046C6
:104B3000FC0000501CFE23A6140040A6160040C630
:104B4000020004609E3F20C71F3C24C7040004608D
:104B500005000460023D84AE833DC4AE103D00A656
:104B6000113D00A6330001001111010011001100D8
:104B700010B5244B1B78012B07D1E12022490001FD
:104B80000A8882420ED2D2180A80204B1A78012A53
:104B900007D100221A70FCF78FF9012801D11C4BB4
:104BA000187010BD00220A801A4A1088411C11801A
:104BB000FA21C900884204D31180174A11780B43A7
:104BC0001370164B19884A1C1A80FA22120191425E
:104BD00005D31A800223104A11780B431370104B2F
:104BE0001A88511C19800F498A4206D90E4A1A8028
:104BF0000423094A11780B4313700122044B1A70E5
:104C0000C3E7C0460011002050010020ED0E002037
:104C1000EC0E0020F810002000080020F610002004
:104C2000F41000201F4E0000204E00000023F0B5BD
:104C300093B00593CD4BCE4A1B780125D9008A1835
:104C40000692CC4A5B009A5ACB4F0792CB4ACC4E85
:104C50008A180892CB4A9A5A0992CB4A8A180A9221
:104C6000CA4A9A5A0B92CA4A8A180C92C94A9B5A43
:104C70000D93C94B0093C94B0193C94B0E93C94B7C
:104C80000F93C94B1093C94B11930E9A009B6C0064
:104C90005B78105B0699079AFFF71CFC0F9A019B43
:104CA00008995B780290105B099AFFF713FC109A41
:104CB0007B780A990390105B0B9AFFF70BFC119A13
:104CC00073780C990490105B0D9AFFF703FC009B1E
:104CD000029A5A70039A019B5A70049B029A7B7045
:104CE0006B4603991B7A70708A4201D26B461B7B1C
:104CF0000499DAB28A4201D26B461B7CDAB2824254
:104D000000D2031CAA4A01375355AA4A013653550B
:104D1000009B013501330093019B01330193062D64
:104D2000B3D1A54B1B78012B49D1A44A00241268AA
:104D30001A4200D06E34A24E00233471910701D57F
:104D40006E2423009F4D00202B71530700D56E3039
:104D50000023F070110701D56E2003000021EB70D5
:104D6000D30600D56E310023B170970601D56E21B0
:104D70000B00AB700023570600D56E33737000260E
:104D8000120601D56E231E006E70002C00D0052483
:104D90008D4A1471002800D00520D070002900D061
:104DA00005219170002B00D0052353700022874B02
:104DB0001D78874BEDB21A80280013B0F0BD854BEB
:104DC00085491B780093854B1B780193009B012B31
:104DD00067D10B78012B00D1CBE16E250026804BEB
:104DE000774A1878957155711571D5709570557011
:104DF00016540522734B9E715E711E71DE709E709B
:104E00005E701D54704B9A715A711A71DA709A70F3
:104E10005A700323734A15782B431370724B1A7818
:104E2000724B1A70724B1A78724B1A70724B1E705A
:104E300002220225654B1A70009B0B706F4B187095
:104E40006F4B1B88002B0ED06E480178A9420AD008
:104E50000223644A1678334313705C4BA94200D393
:104E6000CCE205701D70009B042B0FD1012D01D9E0
:104E7000013DEDB2554B1A78AA4207D01D700223AE
:104E8000614A5570574A11780B4313700123002073
:104E90005E495F4A019C012C00D1B2E2487050701B
:104EA000BDE2009B022B2CD10B78022B08D00122F3
:104EB000584B1A70009B4A4A0B7012784F4B1A706D
:104EC0000022554B01201A70544B554E1A703E4B20
:104ED0003B4D02933B4B36499C46130003920F5CBB
:104EE0007C1EA741039C3C430394019C012C00D1F0
:104EF0004AE1002764466770029C6F7067707770A4
:104F000056E1009B032B00D08CE00B78032B00D1E3
:104F10002FE1334B6E26187800232A4D284AAB71B7
:104F20006B712B71EB70AB706B702E540525937108
:104F300053711371D370937053701654224A009CAE
:104F4000937153711371D370937053701554254D31
:104F50002A7822432A70244A1578244A1570244A54
:104F60001578244A1570244A137061E7D600002092
:104F700038010020EA000020BD10002020010020A0
:104F8000B6100020E400002008010020DE00002010
:104F9000F0000020D8000020CB100020C41000201A
:104FA0005C0F0020BE0F0020A20F0020780F002011
:104FB000D6100020EC100020FD0E0020000F002075
:104FC000370F0020290F0020220F0020F20E0020B2
:104FD000E4100020060F0020E61000200011002041
:104FE000050F0020EB0E002003110020E11000202F
:104FF00001110020E0100020F30E0020040F00201B
:10500000EA100020E7100020450F0020140F0020B8
:10501000080F0020DF100020DE100020DD1000202F
:105020001B0F0020009B042B54D10878CA4BCB4A9D
:10503000042823D00320CA4D2E7830432870C94855
:1050400001260578C8480570C8480578C848057025
:105050000025C8485D710570C748557106706E20FF
:1050600098709070D870D0701871107100989D7100
:105070000870C248C2490078957108700021C8279D
:105080006E26C04D597051706970BF000231BE4C20
:105090004800205AFA24A400A04203D39E709670C0
:1050A000052005E0B8420ED80020987090700020CE
:1050B00068540131013201330529E8D10022B34B94
:1050C00001251A80BCE698780028E9D1907800285C
:1050D000E6D1ECE7009B002B4BD10B78012B02D0E3
:1050E000DA1E012A19D8019B012B12D19C4A0233E6
:1050F0001078034313709C4B1A789E4B1A709C4B8C
:105100001A789D4B1A7000239C4A0B7012789C4BA6
:105110001A7000229D4B1A80D2E6022B00D0CFE6F7
:1051200000229B4B9B481A70019B9B4A012B16D176
:105130009A4B05781B782B43DBB2002B02D11388E6
:10514000002B0CD0884B1D788A4B1D70884B1D7826
:10515000894B1D700323824D2E7833432B7000231F
:105160001380864A037012780B70854B1A700025E5
:1051700066E6009B814A0B701278814B1A70794B5E
:105180001B78012BF3D19BE6764F3F78A74200D1E5
:1051900088E07378002B03D162466E336B705370D6
:1051A0000522029B5A70714B043A1B78DBB20593BF
:1051B000029C013001340294012401360135A444DB
:1051C000062800D08BE6002A02D0754A0598507058
:1051D000039A002A02D00120724A1070019A012A13
:1051E00004D00023704A1380704A13708A784D7877
:1051F0006F48AD18CA78AD180A790121AD186D4A0B
:10520000EDB2157000221600475CBE424CD3BC467E
:10521000974200D294466246D2B201310529F3D1B9
:105220006549B21A0E706549D2B20A704D490978C3
:105230008C466446CFB26249012C7AD1614B1C780E
:10524000012C05D01F70464B1C001B783B4323707C
:10525000564B9C46002E2AD106220E705A48310029
:105260001E7003F035FF06223100584803F030FF6E
:1052700006223100564803F02BFF002D4BD13E4B48
:105280001A78AA4200D1DBE51D700223444A55700A
:10529000334A11780B4313702B1C042D00D90423BF
:1052A000DDB2CDE500272AE632003E00B5E7012A4F
:1052B00019D9012362460B70137000221100042BD0
:1052C00004D83B4AD25CB2420AD00A002248C254F7
:1052D0002248C2542B4AD1540133072BEDD1CCE7DD
:1052E0006E220521F2E700236246137001220B7043
:1052F00000231900042A04D8835C8B4201D06E235A
:105300000521154EB354154EB3541E4B995401321A
:10531000072AEDD1B1E7042D07D9082D07D90C23B1
:10532000AB42AD416D420335A9E73D00A7E7022539
:10533000A5E700220A701C490A80154A1278012A42
:1053400007D1164A1278002A44D1124A1278012A4B
:1053500040D01D00A0E7C046370F0020290F0020D5
:10536000EB0E002003110020E110002001110020AD
:10537000E0100020F30E0020F20E0020050F0020A8
:10538000040F0020220F00205C0F0020E4100020FA
:10539000DF100020E50E0020B20E0020B60E002027
:1053A000450F0020DE100020EA100020D21000205F
:1053B000D6100020D5100020D4100020D3100020DB
:1053C000E810002002110020380F00202A0F0020D2
:1053D000230F00206E200021144A144C5070144AF0
:1053E000A07051709170D1701171124A0531E07046
:1053F000207151709170D1701171AAE70D00197070
:1054000031E54C78002C0AD1084CE45C002C04D126
:10541000074CE45C002C00D141E5092454700133B1
:1054200001310132052B00D034E5C5E4370F0020EF
:10543000290F0020220F00200020704710B55921AD
:1054400016208824044B5A68012A00D110BD5960E7
:1054500058605C60F7E7C046FC000050F8B572B6D3
:10546000FFF7D8FA0421402000F024FDFFF702FAEC
:10547000FFF72CFAFFF7C4F9FFF770F9FFF790F97F
:10548000FFF75CF8FFF772F8FFF788F8FFF79AF874
:10549000494A4A4B1168186800F0C0F900F0E4F975
:1054A00062B600F0F3FC464C05252060FBF744F99A
:1054B000206800F0E5FCFFF7C1FF0023012219007E
:1054C000502000F0B9FD002364263E4C6360FDF7D8
:1054D00029FCFEF76FFAFEF7DBFFFDF763F93A4BA5
:1054E0001A88002A00D11D80384B1A88002A01D161
:1054F000374A1A80374B1A88002A07D11E80FCF7DA
:105500007FFDFCF7C9FA0122334B1A70334B1A881E
:1055100097B2002A0BD1C8321A80FDF729FCFFF799
:105520008DFF01232E4A11680B43136067602D4BDA
:105530002D4A1978572399432C4B1888002937D0C6
:1055400096218900884235D2002111601A88002AEC
:1055500025D1274A1A80274A1388002B0FD0013BF8
:105560009BB21380002B0AD1234A1370234A137075
:10557000234A1370234A033311780B431370FCF74B
:1055800079FCFBF741F8FFF7F3FAFFF755FFFFF758
:105590004DFB1D4B1870FDF70DFBFDF7E1FC1B4BA0
:1055A0001A78012A93D100221A70FBF7C7FB8EE705
:1055B0000128CAD90121C8E7ECAA0000F0AA00001E
:1055C00024110020FC000050121100205201002084
:1055D000B80B000014110020B31000201611002099
:1055E0000040004000080020284200501811002010
:1055F000E7030000120F002000110020F30E00202E
:10560000F20E0020EB0E0020A0080020EC0E00207F
:10561000F0B50E0085B0022102933023534D314086
:1056200004008B4052480431AC4200D07DE0406918
:105630000340CB40012B00D182E00A2149421941AD
:10564000C90700D47FE04B4B1B6801931100019800
:1056500000F0C8FDFF2305250127039000933900C2
:10566000039800F0BFFD80235B0498425FD8424B53
:10567000C3181B0C1A1CDBB2022B00D20222D3B2BD
:105680001900009300F0AEFD80235B0298424ED8D3
:1056900085B2009901987943694300F0A3FD009B0E
:1056A000013D013FAAB2013BFFB2009201900322EB
:1056B000DBB2072F01D8314AD25D80214900206931
:1056C0000842FCD1FF257008C00085408340216856
:1056D000B000A9430B4307218140824023606368E7
:1056E0008B43134363600823F1008B40A26813438C
:1056F000A3601023B34022691A409342FBD00C25CB
:10570000029B75431C34002B1FD1621913689BB296
:10571000136064192368009A1B0C1B042360236820
:1057200001981A43226005B0F0BD806980E77F00D0
:10573000013DFFB2002D00D091E720270E4DA8E7D4
:1057400080231B0281E70E4B7FE7661933680D4902
:105750009BB23360009B3768581C029B584300F093
:1057600041FD0138000438433060D2E700000440B6
:10577000000200505C010020FFFF0000E4AA0000CE
:10578000001BB7001027000001230B408A0702D539
:105790008022520013434A0702D58022520213434B
:1057A000090702D5802252041343826813438360A1
:1057B000704743690B43436170470000F8B505002B
:1057C00000F040FA124B002498421FD1E5277F26B3
:1057D00004343F02281900F035FA431C16D0030C9C
:1057E0000434B343BB420DD1030CD943020AD2B2F5
:1057F000C9B28A4206D1074ADBB212689A4201D97D
:10580000054AD05480239B009C42E3D12000F8BD80
:105810000100AA55281100203411002010B50E4BAC
:10582000802800D980201860FF2180220B4803F0D7
:105830004FFC882459211620094B5A68012A07D1A8
:1058400000F0F8F90823074A11680B43136010BDF4
:10585000596058605C60F0E7281100203411002086
:10586000FC00005000C00050FC2010B50002FFF703
:10587000A5FFFC23002817D1FE200002FFF79EFFA2
:10588000FE23002810D1FC20000200F0A9F9FC2022
:105890000649000200F0FAF9FC2304201B02044A26
:1058A0001360044B186010BD1B02F8E70100AA55F5
:1058B000301100202C1100200123002907D042B212
:1058C000DB18002A03DB034B1B5C0B700023180062
:1058D0007047C04634110020F0B585B06B4601908A
:1058E0001B7901205BB20291002B45DB304B019A02
:1058F0009A5C8A423FD0019A995480222D4B9200A3
:105900001D682B1D934221D92B4B2C4A1B68002765
:105910009C180393631E9C41FE236442640A1B028D
:105920006402E418200000F05BF92000244900F034
:10593000ADF90426234B1B689F421FD33500039803
:1059400000F04EF91C4B1C601A4B1D60019BE521B9
:10595000DB43029ADBB21B021343019A09061604C9
:105960001E43154B31431868281800F08FF9114A6F
:10597000136804331360002005B0F0BD0C4BDA5DF2
:10598000FF2A13D0FF2339021B02591A3B04134389
:105990001943E5231B061943A01900F077F980236A
:1059A000351D08369B009E42C9D82E000137C1E73D
:1059B000341100202C110020301100200004FFFFC2
:1059C0000100AA5528110020084830B5846C084D04
:1059D0002C400C4384640C24816CA14311438164EA
:1059E000826C04490A408264C36430BD00000E40EA
:1059F000FFFBFFFFFFFFFCFFCB0704D50223094A93
:105A0000906C034393640223194203D0054A106D3E
:105A100003431365490704D50223024A516D0B4322
:105A20005365704700000E400D4B00205B6A10B5B7
:105A3000DA0313D4DC04E40F9A0510210134920F29
:105A4000032A01D00749895C3F22074813402033CD
:105A5000584300F0C7FB210000F0C4FB10BDC04656
:105A600000020050F4AA0000001BB700FF239B02B5
:105A700070B518420DD0850A8605EDB2F60EB54018
:105A80000D4C03039B0F1B199B001C68AC43144374
:105A90001C60F0235B0518420DD04300C400C00118
:105AA000240FC00E8440054A9B0F9B189B001A6868
:105AB000A2430A431A6070BD8700001484000014DA
:105AC000054AC30F9B181F2210401E3A82409B00BC
:105AD00019680A431A6070478100001470B5040009
:105AE000114B12491D6800F07DFB114A431C1168DF
:105AF000104A61435160002191600531116080219D
:105B00006B436D085B1949021068084201D1002BF4
:105B100005DC13680B4204D00020106070BD013B0F
:105B2000F2E701204042F9E75C01002040420F000B
:105B30005801002010E000E0064B0749CA68024007
:105B4000824201D1012302E0013B002BF6D1180073
:105B50007047C046C127090000020050F8B5042371
:105B60000F4C0600E56822681020134323600F00E5
:105B7000FFF7E2FF072322691A4322610F22E1693E
:105B800091433943E161206998433043206100F03B
:105B9000A7FA1022154202D1236893432360F8BD6F
:105BA000000200500D4A10B51368040003430120A1
:105BB0001360044201D0FFF7BFFF0220044201D06E
:105BC000FFF7BAFF630702D51020FFF7B5FF0820E3
:105BD000044201D0FFF7B0FF10BDC04600020050E4
:105BE000114B10B50A210400186800F0FBFA2221BD
:105BF0000E4B8200D96021395C601961002A0AD0FD
:105C00001C69013A200008400C42F7D1002A02D05A
:105C10001A68520607D50120054A4042106040220A
:105C200019680A431A6010BD5C01002000C00050D2
:105C3000B41100200123024A11680B43136070471E
:105C400000C000500E4B10B50A210400186800F087
:105C5000C9FA00210B4A8300D160013154601161FF
:105C6000002B05D01069013B0842F9D1002B04D16B
:105C70000120054B4042186010BD9068FCE7C0460B
:105C80005C01002000C00050B4110020104B70B522
:105C900005000C0018680A2100F0A4FA21210D4B20
:105CA0004200D96020395D609C601961002A0AD0E9
:105CB0001C69013A200008400C42F7D1002A02D0AA
:105CC0001B6C5B0603D50120034B4042186070BD7E
:105CD0005C01002000C00050B41100200023F7B583
:105CE000019201249C40214208D003225F00BA4067
:105CF00004689443019ABA40144304600133102BA2
:105D0000EFD1F7BD130E8B401202120A8A4010B574
:105D1000846923438361C3691A43C26110BD0000D3
:105D20007046EFF30881EFF30982024B9847004772
:105D300070470000395D000010B5430700D5110021
:105D40008B69074A1C88944203D0064803F0E4F8A4
:105D5000FEE70024044A023314608B6110BDC04684
:105D6000ABBE0000F7AA000054010020802070B5EF
:105D70000D250B4B8C18C000A14201D1100070BD45
:105D80009E690642FCD100268E570A2E03D11D6063
:105D90009E690642FCD100268E5701311E60EBE75A
:105DA000000005400222044B98691042FCD11B6898
:105DB00001200B707047C04600000540C02270B53E
:105DC0000F4C1203A369050013408022D2029342B4
:105DD0000AD1FFF729FE0B4B9D4207D1E169090F5C
:105DE000013100F0FFF970BD0748F4E7074A0F23BF
:105DF000216A954201D11940F2E70909FBE7C04643
:105E00000002005000001940001BB70000001B40BA
:105E100070B504000E00FFF7D1FF050070080138CF
:105E20003100401900F0DEF9054A431E626041224C
:105E3000010062632800636100F0D4F970BDC046C0
:105E40000180000070B50C000C4B05000A21186899
:105E5000A61800F0C7F98022D200B44204D170BD68
:105E6000431E002804DD18002B6A1342F8D10300FA
:105E70002078013428601800EFE7C0465C0100205C
:105E8000A022D2055368034353607047A023DB056B
:105E900058687047064A030E9B1801220002000A48
:105EA000824019681143196019689143196070475D
:105EB0000800005010B5A024E405626E120B130315
:105EC0000B430343636610BD7FB56946124B6A46B8
:105ED00070CB70C11B680B60104B1149984208D100
:105EE0004B695B055B0F032B13D89B00D05804B0A4
:105EF00070BD0C4B984202D14B695B04F2E70A4C2F
:105F000007238969A04202D1090A0B40EBE7090B7C
:105F1000FBE70648EBE7C04608AB00000000014085
:105F2000000200500001014000001140001BB700BA
:105F3000F7B5050017000191FFF7C6FF4608BE42FE
:105F40001CD380239B04984210D303248608390075
:105F5000300000F047F901003000019BA9606C603F
:105F600001342B60614300F03DF9FEBD8023012424
:105F70005B049842EBD206000024E8E700240221EB
:105F8000EBE7C3680B43C36070470000F0B585B012
:105F90000E0069461B4B050091CB91C103206A4658
:105FA0001B680B6018494B69CC6903409B002405B2
:105FB0009858240F0134002801D100F049F821003D
:105FC00000F010F90023AB6303330400AB60002E34
:105FD00014D070083100001900F004F98023013852
:105FE0005B0298420CD3F0003100001900F0FAF87F
:105FF0008023000901381B0603436B6205B0F0BD26
:106000006862FBE718AB00000002005070B5802505
:1060100003008C18AD00A14205D1100002E0013848
:10602000002802D170BD8020C0059E692E42F6D0A6
:10603000087801311860EEE79B0003430B435200E0
:10604000134308221343014A136070470040004085
:106050000D4B00205B6A10B5DA0313D4DC04E40FA7
:106060009A0510210134920F032A01D00749895C57
:106070003F22074813402033584300F0B3F8210073
:1060800000F0B0F810BDC0460002005028AB000080
:10609000001BB700072310B50D4C206918400228DB
:1060A00010D0032811D0013843425841094B4042D7
:1060B0001840094BC0180F23E1691940013100F065
:1060C00091F810BDFFF7C4FFF5E70448F3E7C046B9
:1060D00000020050006549FF001BB70010270000B8
:1060E00010B5FFF7D7FF054B05491860054B064C67
:1060F000C01800F077F8206010BDC0465C01002099
:1061000040420F0020A107005801002010B503F005
:1061100073F8582303600120404210BD10B503F00E
:106120006BF8582303600120404210BD10B503F006
:1061300063F858230360002010BD10B503F05CF82D
:10614000582303600120404210BD00000B490C4A57
:106150000C4B9B1A03DD043BC858D050FBDC0A48AB
:106160000A4901600A4901600A4901600A480B496D
:10617000016005480A490160F9F7F4FFF8AB000037
:10618000000000209407002000010050590000008A
:10619000160000008800000060000050A55A0000B2
:1061A00000000000FEE7C04602B4714649084900FD
:1061B000095649008E4402BC7047C04602B471467D
:1061C00049084900095C49008E4402BC7047C0463A
:1061D00003B47146490840004900095A49008E44F9
:1061E00003BC7047002243088B4274D303098B42DF
:1061F0005FD3030A8B4244D3030B8B4228D3030C97
:106200008B420DD3FF22090212BA030C8B4202D338
:106210001212090265D0030B8B4219D300E0090A60
:10622000C30B8B4201D3CB03C01A5241830B8B4269
:1062300001D38B03C01A5241430B8B4201D34B0352
:10624000C01A5241030B8B4201D30B03C01A5241B7
:10625000C30A8B4201D3CB02C01A5241830A8B423C
:1062600001D38B02C01A5241430A8B4201D34B0225
:10627000C01A5241030A8B4201D30B02C01A524189
:10628000CDD2C3098B4201D3CB01C01A524183093D
:106290008B4201D38B01C01A524143098B4201D377
:1062A0004B01C01A524103098B4201D30B01C01AA2
:1062B0005241C3088B4201D3CB00C01A524183081C
:1062C0008B4201D38B00C01A524143088B4201D349
:1062D0004B00C01A5241411A00D2014652411046A9
:1062E0007047FFE701B5002000F0F0F802BDC0469E
:1062F0000029F7D076E7704703460B437FD400228E
:1063000043088B4274D303098B425FD3030A8B4249
:1063100044D3030B8B4228D3030C8B420DD3FF22B3
:10632000090212BA030C8B4202D31212090265D081
:10633000030B8B4219D300E0090AC30B8B4201D334
:10634000CB03C01A5241830B8B4201D38B03C01A7B
:106350005241430B8B4201D34B03C01A5241030BF2
:106360008B4201D30B03C01A5241C30A8B4201D3A3
:10637000CB02C01A5241830A8B4201D38B02C01A4E
:106380005241430A8B4201D34B02C01A5241030AC5
:106390008B4201D30B02C01A5241CDD2C3098B42AA
:1063A00001D3CB01C01A524183098B4201D38B0127
:1063B000C01A524143098B4201D34B01C01A5241CA
:1063C00003098B4201D30B01C01A5241C3088B420F
:1063D00001D3CB00C01A524183088B4201D38B00FA
:1063E000C01A524143088B4201D34B00C01A52419C
:1063F000411A00D201465241104670475DE0CA0F73
:1064000000D04942031000D34042534000229C4632
:1064100003098B422DD3030A8B4212D3FC2289013C
:1064200012BA030A8B420CD3890192118B4208D312
:10643000890192118B4204D389013AD0921100E074
:106440008909C3098B4201D3CB01C01A5241830988
:106450008B4201D38B01C01A524143098B4201D3B5
:106460004B01C01A524103098B4201D30B01C01AE0
:106470005241C3088B4201D3CB00C01A524183085A
:106480008B4201D38B00C01A5241D9D243088B42B0
:1064900001D34B00C01A5241411A00D20146634653
:1064A00052415B10104601D34042002B00D54942B7
:1064B000704763465B1000D3404201B5002000F0F6
:1064C00005F802BD0029F8D016E770477047C046AE
:1064D000844608006146FFE71FB500F009FC00286C
:1064E00001D40021C8421FBD10B500F085FB404219
:1064F000013010BD10B500F0FBFB002801DB0020CF
:1065000010BD012010BDC04610B500F0F1FB002801
:1065100001DD002010BD012010BDC04610B500F007
:1065200097FB002801DC002010BD012010BDC046F3
:1065300010B500F08DFB002801DA002010BD01200D
:1065400010BDC0469E2110B5C905041CFFF7F0FF21
:10655000002803D1201C00F0AFFF10BD9E21201C9D
:10656000C90500F05FFD00F0A7FF80231B06C018DF
:10657000F3E7C046F0B5C64647027B0A9C464B028D
:106580005A0A904645004A002D0E120ECE0F00B555
:106590009909C40FBF09AB1AB4424BD0002B39DDA7
:1065A000002A00D177E0FF2D00D1C1E08022D20483
:1065B00011431B2B00DCFFE0013F7A0100D4B1E066
:1065C00001277F42BF01BA091600100002F010FB3C
:1065D000330005388340854200DCD5E0B94F2D1AE1
:1065E0001F405A0700D178E10F221340042B00D13D
:1065F00073E104377B0100D46FE1681CFE2D00D0ED
:106600007DE0FF200022C0051043E407204380BC4A
:10661000B846F0BD002B46D0531B002D73D1002F80
:1066200000D139E1012B00D17EE1FF2B00D156E1F1
:10663000013B6EE0002B00DC85E0002A51D10029EF
:1066400072D05A1E012B00D12CE1FF2B70D01B2AD7
:106650004CDC130008002022D840D31A99400B00CC
:106660005A1E93410343FF188023DB041F4200D1CD
:106670002CE10135FF2DC4D0934A79081140012245
:1066800017400F437A0700D08DE01F42B5D1FB08B9
:106690009C462B002EE0002946D0012B67D0FF2B13
:1066A00046D0013B85E7FE206A1C104200D099E0ED
:1066B000002D00D0E6E0002F00D12FE1002919D0F5
:1066C00080257A1AED042A4200D15AE13400CF1B0A
:1066D00000D18FE001202F4212D1FB089C460023FD
:1066E00008E0FF2D24D01B2B00DC9AE00537FB08C7
:1066F0009C462B0062465202520AD8B283E7C0B2CF
:10670000BA01520A7FE7FF2A00D1E8E08020C004E6
:1067100007431B2B00DC88E04F1E34001500790175
:1067200000D54DE72B000437FA089446FF2BE1D142
:106730006346002B00D145E18022D2031A43520266
:10674000FF20520A5FE7002B57D0531B002D78D152
:10675000002F00D1A1E05D1E012B00D1A2E0FF2B94
:1067600000D1BDE01B2D00DDC0E02B0070E0791AE8
:106770004A0100D4B6E089018D09280002F038FAF8
:106780002B000538834001252022401B0130121ABE
:106790001F009340C7405A1E93411F432AD0002533
:1067A0007B0700D108E10F233B40042B00D020E7FA
:1067B0007B0100D521E76AE708002022D840D31AE0
:1067C00099400B005A1E93410343FF1A7B0100D5E9
:1067D000F8E67B0700D15AE70F233B40042B00D09B
:1067E00007E754E77B1A1A005B0158D4002A00D04F
:1067F000EAE600240020002205E7FE226B1C1A4274
:1068000031D1002D77D1002F00D1A6E0002900D191
:10681000BCE07A18530100D4BAE092010120520A78
:10682000F1E68022D204114314E738002024D84036
:10683000E31A9F407B1E9F41074334001500CF1B86
:10684000C4E7FF2A4CD01B2B50DC8020C004074338
:1068500038002025D840EB1A9F407B1E9F410743FC
:1068600015007F1800E7FF2B00D1CAE67F187F08CC
:106870007A0700D190E00F223A40042A00D18BE041
:10688000043751E7002F5DD1002900D086E0802237
:106890000024FF20D203B6E634000F0044E73400A2
:1068A000CA1B91E67B185A0100D47EE0064F5B08B4
:1068B0001F405A0758D00F221340042B54D00223F4
:1068C000043731E7FFFFFFFBFFFFFF7D7B0704D0AD
:1068D0000F233B40042B00D08BE62B0024E7340031
:1068E000C44625E7CB089C46012303E70531CB08C6
:1068F0009C461300FEE6002FF2D0002936D08023FC
:10690000DB039C4502D3984500D2C44680226346EF
:10691000D2031A435202FF20520A74E6002900D122
:1069200067E73400C446E5E6CB1B5A0124D59B013A
:106930009C09200002F05CF92300053883403400F4
:10694000013521E7002911D08023DB039C45DDD3ED
:106950009845DBD23400C446D8E7002900D149E786
:10696000CB089C460023C5E6022590E680226346BC
:10697000D203FF201A4346E6DB089C46340001237D
:10698000B8E6002A15D1002400203CE60023B1E639
:10699000D3089C460023ADE61D0078E680224346DE
:1069A000D2033400FF201A432DE6DB089C46012366
:1069B000A0E6D20894469DE601207B0100D59EE624
:1069C0003900CDE7FF201A001DE6C046F0B54F465E
:1069D0004646D6464502C0B5C30F470099460E1C31
:1069E0006D0A3F0E5AD0FF2F21D08023ED00DB042B
:1069F0001D43002398469A467F3F74027300640A41
:106A00001B0EF60F002B1FD0FF2B42D08022002040
:106A1000E400D20414437F3B4A46FF1A43467240C7
:106A20000F2B00D99CE071499B00CB589F46002D4D
:106A300059D108239846063B74029A467300640AAB
:106A40001B0EF60F002BDFD1002C3BD101234A4651
:106A50004146724019430E2918D8654889004158AB
:106A60008F465346022B00D1B9E0032B6ED04A4625
:106A70002C00012B40D100200024C0052043D20768
:106A80001043E0BCBA46B146A846F0BDFF20002442
:106A9000F3E7002C20D10223FF3FD8E7002D05D1DA
:106AA00004239846033B00279A46A6E7280002F0F5
:106AB0009FF87627431F9D4000237F4298469A46C1
:106AC0003F1A9AE7200002F093F8431F9C40762378
:106AD0005B421B1A00209FE7032342461A4390465D
:106AE0000320FC3398E70C239846093BFF279A467E
:106AF00083E703282CD0320038007F30002847DDA0
:106B0000630704D00F232340042B00D00434230157
:106B100003D53800374B80301C40FE28B6DCA4017A
:106B2000640AC0B2A9E780240022FF20E403A4E79E
:106B30008023DB031D4201D01C420BD08024E403E0
:106B40002C4364024A46FF20640A96E74E462C0016
:106B50008023DB031C4364023200FF20640A8CE7BD
:106B60006D01600185422ED21B230024013F0126C6
:106B7000290064006D00002901DB854201D32D1A34
:106B80003443013B002BF3D16B1E9D412C43B3E7F3
:106B900003001A3300DA6EE7012321001B1A9E3727
:106BA000D940BC400B00611E8C412343590704D0DF
:106BB0000F211940042900D00433590113D49B013B
:106BC00000205C0A59E71A2301242D1ACFE7981EEA
:106BD00043425841404232000024C0B24DE74A4689
:106BE000FF20002449E70120002446E72CAB0000E9
:106BF0006CAB0000FFFFFFF730B543024200C50F4A
:106C000048025B0A440A48009C46120E000EC90F57
:106C1000FF2A11D0FF280CD0012382420AD1A445BB
:106C200008D18D4211D0002A04D163465A1E9341E7
:106C300000E00123180030BD0123FF28FAD162468D
:106C40002243F7D12B004B40F4E70023F2E7C04684
:106C500043025B0A42009C46C30F480210B5440A37
:106C60004800120E000EC90FFF2A1AD0FF280BD0C1
:106C7000002A24D1624600281ED1002C2ED0002AE2
:106C800032D1480001380BE0002C2AD1002A02D171
:106C90006246002AF5D08B421DD001205B4218438A
:106CA00010BD6246002A1CD1FF28F6D1002C18D155
:106CB00020008B42F1D1F3E7002AE2D0EBE7002875
:106CC000EBD08B42E9D18242E7DC04DBA445E4D877
:106CD0000020A445E4D258000138E1E7002ADFD0C3
:106CE000DBE702204042DBE78B42D6D1EEE7C0462D
:106CF00043025B0A42009C46C30F480210B5440A97
:106D00004800120E000EC90FFF2A15D0FF280BD025
:106D1000002A1AD1624600281DD1002C22D0002A58
:106D200032D1480001380FE0002C0CD1002A14D1D8
:106D30006246002AF5D010E06246002A03D1FF28FF
:106D400005D1002C1CD0022010BD00280DD101203F
:106D50005B421843F8E7002AE3D08B42F7D1580092
:106D60000138F1E7002AEFD0F1E78B42EFD1824200
:106D7000EDDCF4DBA445EAD80020A445E4D2EEE73C
:106D800020008B42E3D1DFE78B42E0D1F2E7C0463F
:106D9000F0B54646D6464F464402C0B5C30F46003E
:106DA00098460D1C640A360E00D1CBE0FF2E6ED043
:106DB0008023E400DB041C43002399469A467F3E6F
:106DC0006F026B007F0A1B0EED0F002B6DD0FF2BA7
:106DD00000D1A6E07F3BF6184B460A2B00DD82E08F
:106DE0008023FF00DB041F4343466B4098464B461D
:106DF0000022022B0FDD494601238B40A621C9004A
:106E00000B4200D06FE0902189000B4200D0D3E00C
:106E10008821194264D1200C2404240C21003B0C4D
:106E20003F043F0C79435C4347435843E4190B0C40
:106E30001B199F4202D980225202801809041A04A9
:106E4000090C52189401611E8C411B0C920E1B18E8
:106E500014439B011C431B0100D5CDE030007F3063
:106E6000002800DCAEE063070BD00F233200234084
:106E7000042B06D00434230103D580321000684B64
:106E80001C40FE2866DCA3015B0AC0B21EE0002C99
:106E900000D08BE008239946063B6F029A466B00B0
:106EA0007F0A1B0EED0F002B91D1002F61D14A46B6
:106EB00001231A4391460A2A15DC43466B40984643
:106EC0004B460122022B96DC00200023C00518430C
:106ED0004346DD072843E0BCBA46B146A846F0BDAC
:106EE000A8463C0092465346022B33D0032B11D0C8
:106EF000012BE9D030008030721C002863DD63076D
:106F0000B9D00F232340042BB4D1B4E70F2A78D093
:106F1000A8463C008023DB0323435B02FF205B0A7F
:106F2000D4E7FF36002F2FD102234A4613430A2B02
:106F3000D9DC42466A4090464A46002A0AD0994621
:106F4000022258E7002C08D104239946033B00266F
:106F50009A4635E7FF200023B8E7200001F048FEFD
:106F60007626431F9C400023764299469A46361A5D
:106F700026E7380001F03CFE4B46361A763E0A2BD7
:106F8000B1DC053887402FE703234A461A43130034
:106F90000A2ABBDC42466A40904601229A40882178
:106FA00013000322194200D135E799E70C239946D3
:106FB000093BFF269A4603E7002398468023FF20DB
:106FC000DB0383E7320003001A3300DA7CE79E32EA
:106FD0000123210094401B1AD940621E94410C43A6
:106FE000630704D00F232340042B00D00434630133
:106FF00011D50120002369E7012362081C401443D6
:1070000078E78023DB031C4284D01F4282D1A8464C
:10701000FF203B435AE7A30100205B0A56E7C04626
:10702000FFFFFFF7F0B5C64647027B0A4A0245005C
:107030009C46C40F530A4800984600B52D0EBF0960
:10704000000ECE0F9209FF2800D171E001235E40AF
:107050002B1AB4423CD0002B00DC9CE1002800D16C
:10706000A3E0FF2D00D18BE08021C9040A431B2B34
:1070700000DCFBE0013F7B0100D47BE001277F4285
:10708000BF01B9090E00080001F0B2FD3300053858
:107090008340854200DCD2E0B44F2D1A1F405A07CE
:1070A00000D1F6E00F221340042B00D1F1E00437A9
:1070B0007B0100D4EDE0681CFE2D00D090E0FF20A5
:1070C0000022C0051043E407204380BCB846F0BD51
:1070D000002B00DC77E100286FD1002A4CD0591E2C
:1070E000012B00D146E1FF2B4AD01B296ADC0B00A3
:1070F00011002020D940C31A9A40531E9A410A43D6
:10710000BF188023DB041F4200D1BBE00135FF2DF7
:10711000D5D0974A79081140012217400F437A07CA
:1071200000D09AE01F42C6D1FB089C462B004DE0E0
:107130002B00FF3B002A2ED101214E40B44200D14A
:10714000B4E0002B50D0002D00D0EAE0FF23002F48
:1071500000D1FAE0591E012B00D15CE1FF2B00D1D8
:107160003DE11B2900DC22E1571E340005007B01B4
:1071700000D583E72B000437FA089446FF2B25D16E
:107180006346002B9BD080226346D2031A435202EF
:10719000FF20520A95E7B44200D1A4E0002B23D08F
:1071A000002DD3D0C4463400EDE7002AE4D0012BF3
:1071B00039D0FF2BE4D0013B59E7FF2DE0D01B2B4A
:1071C00000DCA6E00537FB089C462B006246520215
:1071D000520AD8B275E701203A007B0100D43FE1A2
:1071E000C0B2BA01520A6CE7FE216B1C194252D19F
:1071F000002D00D0ACE0002F00D11AE1002A00D110
:10720000F4E08021BB1AC9040B4200D13CE1012407
:10721000D71B3440002F46D001200F42E1D1FB089C
:107220009C460023D2E7BF1A7A0100D4DAE0BD0100
:10723000A80901F0DDFCAB090538834001252022B7
:10724000401B0130121A1F009340C7405A1E934141
:107250001F4328D000257B07BDD00F233B40042BC4
:1072600000D024E77B0100D525E75DE71100202051
:10727000D940C31A9A40531E9A410A43BF1A7B0150
:1072800000D5FDE67B0704D00F233B40042B00D044
:107290000DE72B0070E7BB1A19005B0162D40029CF
:1072A00000D0EFE60024002000220AE7002B1CD0CB
:1072B000002D00D003E7FF23002F47D0591E012BDC
:1072C00058D0FF2B00D18BE01B2900DD90E00B0094
:1072D00039002025D940EB1A9F407B1E9F410F4368
:1072E0000500BF180DE7002B17D1FE216B1C1942BA
:1072F0001BD1002D00D080E0002F00D1AEE0002A8D
:1073000074D0BA18530100D4AAE092010120520AA5
:10731000D7E68021C9040A43EAE6002DCBD0C44653
:1073200031E73400FF200022CBE6FF2B00D1C6E678
:10733000BA185208510705D00F21171D1140042912
:1073400000D019E7D208944640E73400170013E74D
:10735000002F75D1002A00D09DE080220024FF205C
:10736000D203AEE60124D11B34408BE6FFFFFFFBC6
:10737000FFFFFF7DBB185A0100D494E04D4A5B0823
:107380001A40590700D192E00F210B40042B6ED018
:107390000223171DF0E6002B00D125E7411B0B004F
:1073A000002D00D1D3E68023DB041F43D9E63B0048
:1073B0002024CB40611A8F40791E8F411F43340037
:1073C0000500D71B5BE7002B8FD0431B002D00D19E
:1073D00072E71B2B0CDC8021C9040F4378E73400D3
:1073E000C446CDE6FB089C460123EFE60023EDE60C
:1073F0000532D3089C460300E8E6002FF0D0002AAF
:1074000037D08023DB039C4500D2BCE6984500D3EF
:10741000B9E6C446B7E6D31B5A0130D59B019C0997
:10742000200001F0E5FB23000538834034000125EE
:1074300005E7002A18D001240023C4463440C5E6DD
:10744000002A16D08023DB039C4500D29BE698459A
:1074500000D398E60124C446344094E6002A04D0C0
:10746000D3089C460023B1E60024002029E6023B15
:1074700068E780226346D203FF201A4321E6DB0837
:107480009C4634000123A1E6002B00D10AE7DB086B
:107490009C4600239AE6802243460124D203FF2023
:1074A0001A4334400DE6DB089C4601238EE6022396
:1074B00048E7C046FFFFFF7D41024200C30F490A73
:1074C0000020120E7E2A03DD9D2A02DD094A98184B
:1074D0007047802000040143952A07DC9620821A19
:1074E000D1404842002BF3D10800F1E7963A914091
:1074F000F7E7C046FFFFFF7F70B5002813D0C31722
:10750000C5185D40C40F280001F072FB9E230100E6
:107510001B1A07280EDD082830D008398D406D026F
:107520006D0AD8B201E000240025C0052843E40715
:10753000204370BD042816DD052801D0421F954068
:10754000104A2A4068070AD00F202840042806D095
:107550000432500103D50B4B1A409F235B1A920152
:10756000550AD8B2E1E7020028001B329040421EC3
:1075700090410522521AD5400543E1E76D0296205D
:107580006D0AD2E7FFFFFFFB10B504000020002CBE
:107590000ED0200001F02CFB03009E20C01A072B08
:1075A00009DD082B2CD0083B9C406402640AC0B261
:1075B000C005204310BD042B16DD052B01D05A1F3A
:1075C0009440114A224061070AD00F21214004292A
:1075D00006D00432510103D59F200B49C01A0A403E
:1075E0009201540AC0B2E3E71A0021001B32914015
:1075F0000A00511E8A410521C91ACC401443E0E714
:1076000064029620640AD3E7FFFFFFFBF0B547460C
:10761000CE4680B583B0009001910E034D000199D4
:107620005F00CC0F710A009E6D0D760F0E4300991E
:1076300000920193C8001903019B7F0DDB0F9C464C
:107640004B0A0099490F1943009BDB009846EB1B3E
:10765000644565D0002B14DD002F00D0AEE00F0094
:107660004246174300D14DE15A1E012B00D1C9E219
:10767000AF4FBB4200D121E2382A00DD58E21300AF
:1076800061E1002B00D1A9E07B1B002D00D0D7E1E8
:107690003400044300D18AE25C1E012B00D125E3B3
:1076A000A34DAB4200D1CFE2382C00DC7FE3424651
:1076B000013A9146904592418E1864461D0032026F
:1076C00061D501235B4299469A4E300001F090FA51
:1076D0000300083B484620210700CA1AD7409E40B5
:1076E00098403A00814632430600AB4200DADDE1C1
:1076F000581B33000130091A8B40C6405D1EAB4158
:1077000017008F4033431F43C2403B001600134312
:1077100000D117E27B0700D05FE1A446380082E089
:10772000002B00DCCCE0002F00D08AE00F004246A6
:10773000174300D1E6E05F1E012B00D146E27C4AF0
:10774000934200D1BAE1382F00DCE0E2421C9146BE
:10775000802212041D00164215D01600744B01350C
:107760009D421DD0744A012116404A4653081140DB
:10777000F7070B431F4376085B0709D00F23B94671
:107780003B40042B04D04B461F1D4F459B41F61A2E
:10779000330200D487E0664A0135954200D085E087
:1077A0002B00002600271B053343E4072343380042
:1077B000190003B0C0BCB946B046F0BD5C4FBD4235
:1077C00000D12EE2382B00DCBAE0431E9842804103
:1077D00036189946330200D573E7D4E7574F6B1C30
:1077E0003B4200D04EE133000F00424603431743B3
:1077F000002D00D0E0E1002B00D119E2002F00D1D4
:107800001CE2821A9042AD41731A5B191D0200D42A
:10781000E3E24346181A8045924107008E1BB618D2
:10782000374300D1F1E2644607000123310080466E
:1078300032023DD443464F07DA0817430023CD08F0
:10784000F9E03B4FBD4200D138E1382B00DD53E178
:1078500080273F0439431F2B00DD02E22027FA1A5C
:107860000F00944697404246DA401743B9466246B5
:10787000474697403A00D940571EBA414F467618BE
:107880003A431318834280419946361A330200D591
:1078900064E74A46530700D1BBE20F231340042B91
:1078A00000D070E74F462B00F8082CE06B055B0D0D
:1078B000214AFF081640720776021743360B72E71B
:1078C000002B00D194E07B1B002D00D01DE1350082
:1078D000054300D14EE25D1E012B00D13BE2144A6C
:1078E000934200D1D0E1382D00DC8CE242460132D7
:1078F0009146802212041D001600114200D02DE78F
:107900000E0040E7C00872071043094AF508934289
:1079100000D08BE107002F4307D0802636032E438B
:1079200036030700024B360B3DE70026004B3AE7D3
:10793000FF070000FFFF7F00FFFF7FFFFE07000043
:1079400080273F0439431F2B00DDBCE02027FA1AB3
:107950000F00974094463A004746DF403A4391462D
:107960004746624697403A00D940571EBA414F46B3
:10797000761A3A43831A9842804199463618330260
:1079800087D57602760A002E00D09EE6484601F0A2
:107990002FF9030018331F2B00DC9BE64A460838FA
:1079A00082409D4200DDA1E05B1B581C1F2800DCCB
:1079B0000FE217001F3BDF40202805D040231B1A91
:1079C0009A40531E9A411743002F6CD00723190089
:1079D000B84639403B4200D12CE70F233B40042BF3
:1079E00000D03BE10025033B320200D560E75AE7B7
:1079F000C84F6B1C3B4200D0B3E033000343002D63
:107A000000D055E10F0042461743002B00D1C9E1D9
:107A1000002F00D112E18218824280417618361A76
:107A2000330200D5E0E1170037433CD00023D208F1
:107A300077071743F5082E035B05360B5B0DB2E69F
:107A4000B54CA74200D1FFE0382B7EDC8024240413
:107A500026431F2B00DD1DE120253400ED1A020016
:107A6000A840AC40DA40451EA841DE401443204304
:107A7000891B43461B1A98459241994664463D002E
:107A80008E187CE74346C71AB946B842BF41731AFD
:107A90007F42DB1B1F0200D580E04F461E001F43C4
:107AA00000D070E70024002300267CE69B4EED1AF0
:107AB00016400200430700D0EFE6F3E67207C00865
:107AC0001043F50826E71F000A00203FFA409446BD
:107AD000202B05D04027FB1A994043460B4398467C
:107AE0004246531E9A4163461A4343E7EB1A8B4DB5
:107AF00015406F07ED089EE7431C994680231B0441
:107B00001E4200D13FE61E0028E6834DAF4200D161
:107B1000BAE0382B00DC03E1434601339946802369
:107B20001B043D001E00194200D017E60E002AE695
:107B3000421E90428041361891461D00320200D507
:107B4000BFE520E6002700262DE64346013B984589
:107B500092418E18994664463D00330200D5B0E547
:107B600011E66D4DAB4200D11BE6424682188242BF
:107B700080417118091AC8075208104381464E08FF
:107B8000520700D148E10F221D000240042A00D014
:107B9000F9E5C208770717430D094CE743461B1A5E
:107BA000984592418E1B99466446B618EBE64246CC
:107BB00064460E00D008A6E6002B00D0DEE0002FC1
:107BC00042D180260024544B3603ECE583188342CF
:107BD000804175182D1A2A0200D4C5E04F4A5B086F
:107BE0001540EA071A4369085B0700D119E10F2322
:107BF0001340042B00D100E1171D9742B641022526
:107C00008E1B50E64346C21A90428041761A3618BF
:107C10009146330220D4D30877071F43F508012388
:107C200009E7C00873071843F50873E6070002E781
:107C3000002F00D136E764460E004046C0087707A3
:107C400000230743F508F6E643464807DA0864468A
:107C50001043CD085EE66446012592E6B94600254C
:107C600091E51F000A00203FFA409446202B05D0E2
:107C70004027FB1A994043460B4398464246531E01
:107C80009A4163461A43FCE543464807DA08104325
:107C9000CD083FE61C003500203CE540202B03D0FA
:107CA0004024E31A9E403043431E98412843E0E6B7
:107CB000002BE9D07307C008424618430B00F508B3
:107CC000134300D126E680231B031D4206D0CE08B5
:107CD0001E4203D13500D00849070843430FC000B6
:107CE000ED00C0085B071843ED0813E643461B1A76
:107CF000984592418E1BB618994619003302AAD4B2
:107D0000CB0877071F4364460123F50893E63B0041
:107D1000A1E5C046FE070000FF070000FFFF7FFF50
:107D200080252D042E431F2B43DC2025EA1A350025
:107D3000944695400200DA40154362469040DE408A
:107D4000421E904189192843404440459241814652
:107D50003D008E1A9AE5030043444345924175184D
:107D6000AD1A2A0200D539E76F07DB081F43ED087B
:107D7000012360E642460E00D008C4E5C008730740
:107D80001843F508002F00D1C4E580231B031D42D2
:107D9000A4D0CE081E42A1D1D008490764463500C0
:107DA00008439BE7002F00D044E50026FBE42300B6
:107DB0004FE61D003200203DEA409446202B03D0C0
:107DC0004025EB1A9E403043431E984163461843BA
:107DD000BAE720210023091A92E4170010001E00C0
:107DE0001F4300D02AE75DE6114BD2081E407707FB
:107DF000760201231743360BD5E4D708490702233F
:107E00000F432D0917E62B008DE76446002300265B
:107E1000C9E42B00D00876E57707C20817430D099F
:107E200009E6D208490711430F0002232D0902E693
:107E3000FFFF7FFFF0B54546DE4657464E4604003D
:107E4000E0B50D0089B0009401951F00019B16005C
:107E50001B03190B019A019BD20F5B0080460C009B
:107E600093465B0D00D1C1E08E4A934234D0009C12
:107E7000019DC900620F0A43802109041143E200F9
:107E80009046894A00249B189A4600230391009348
:107E90003B03190B7A0030008946520DFD0F002A72
:107EA00000D17FE07F4B9A426ED0C900730F0B4325
:107EB00080210904194389467B49F3005218514631
:107EC0008A1A924600215E466E400F2C00D9FBE0D4
:107ED000764AA400125997460A0000990A43039271
:107EE00000D0B7E09A460223904608240093CFE7DB
:107EF0002E0000210023002288461B051343F607AD
:107F000033434046190009B0F0BCBB46B246A9460F
:107F1000A046F0BD039B5D46994643460099022961
:107F200000D1F5E1032900D1A1E00129E0D05446B8
:107F30005F4AA4180494002C00DCFAE15A0704D02C
:107F40000F221A40042A00D076E22E00DA084946B1
:107F5000CB0107D5574B1940894680215346C900AC
:107F60005B180493544B0499994208DC4846430734
:107F70001343984642024B05120B5B0DBDE70021EF
:107F800000228846474BB8E752460B004B49334323
:107F900052189246002B58D102221443002202218B
:107FA000914690E70B00334349D0002900D19EE170
:107FB000080000F01DFE0B235B429C460200844437
:107FC00011004846083988401D23814660461B1A27
:107FD0003000D840030048460343994633008B40A5
:107FE000374952445218924600216CE70A00009922
:107FF0000A4303921CD0002C00D168E1200000F05D
:10800000F7FD02000B381D231B1A009811002500F4
:10801000D84008398D4003002B430393009B8B40CD
:108020009846284B00249B1A9A46002300932FE77A
:10803000002398469A4601330424009328E701223E
:1080400014430022012191463DE7032303211C43F1
:10805000330038E79A460323039400930C2417E770
:1080600000238022984600260E4B120345E780220B
:10807000494612030A43120398462E00094B120B7D
:108080003BE7802203991203114202D04946114274
:10809000F0D08022039B12031A4312035E46014B69
:1080A000120B2AE7FF07000001FCFFFFA8AB00004E
:1080B000FF030000FFFFFFFEFE07000001F8FFFFC7
:1080C000F30300000DFCFFFF0399894500D2F5E0A2
:1080D00000D1F0E05246013A9246002244469046D2
:1080E00003984A461F0E120217431B0203933B04D8
:1080F000110C1B0C00938B46FEF7FAF8009A0B0448
:108100004243210C050019438A4207D9C919013D90
:108110008F4203D88A4201D9851EC919881A594647
:10812000FEF7E6F8009A240442430904240C0300F5
:108130000C43A24204D9E419013BA74200D8F2E063
:108140000399A01A2D040C0C09041D43090C2A0CD8
:108150002B04A9460D001B0C5D430791634351435B
:10816000069462435B182C0CE318994202D98021D3
:1081700049025218190C2D041B042D0C8A185D1984
:10818000904200D284E000D17FE043465D1BAB42C9
:108190009B415446801AC018AD4BE41804948742A2
:1081A00000D1FBE05946FEF7A3F80200009B0590C2
:1081B0005A430B04290C19438A4209D9431EC91991
:1081C00005938F4204D88A4202D9831E0593C919A8
:1081D000881A5946FEF78CF80A04944603002A04CC
:1081E00065460099120C59432A43914207D9D21986
:1081F000013B974203D8914201D9831ED219521AEA
:1082000005990798090405000B43190C8C461904BD
:10821000090C4D4388466146AB466546484306997E
:108220004D43AC46454669435D4609182D0C491936
:10823000884202D98020400284445D46080C2D0407
:1082400009042D0C60444D19824211D30DD0012236
:108250001343804A92456DDB1A1D9A429B41D20816
:108260005B42CC469C44E14671E6002D00D193E090
:10827000591EBA188C46BA4200D285E0824200D21A
:10828000C4E000D1D1E00B00E1E7A84500D37CE7D2
:108290004B46013B04934346039C1B199846A3425B
:1082A0009B41FB1AC018874238D282427DD87AD0CF
:1082B000049B994669E7434500D90BE74146039A79
:1082C000D40750084A081443CA07904609E700F04B
:1082D0008FFC02000300153020321C2800DC92E6DF
:1082E0000099083B994000230391984699E600F0D5
:1082F0007FFC15239C4684440200634620321C2BDD
:1083000000DC5DE63100083881400023894667E6DD
:1083100000212E00002288464F4BEEE58742C7D150
:108320004445C5D8C1E7A24200D809E7831EE41935
:1083300006E72E002200373200DADAE522001E328C
:108340003FDB4D46012250464449121B40181C0099
:10835000290083408140D440581E8341D5402143A9
:108360000B432A00590708D00F211940042904D0D3
:10837000191D99429B41EA1A0B00110263D5002195
:10838000012300228846B8E50B00824200D05EE758
:10839000039A954200D05AE73500CBE5002C41DD29
:1083A000002201235DE7454582D94B46023B9946B1
:1083B000434603995B1898468B429B41FB1AC018B1
:1083C000E3E648461F2201005242121BD1401F34EF
:1083D00004D05246224C1219904003435A1E934136
:1083E00007200B43010000221940184209D00F2139
:1083F000194004291ED0181D9842894103004942A2
:108400004907DB080B439846002376E50399023BB6
:1084100049008C4603998C458941791A5218614666
:108420000391B2E701235B4284E70399A942EDD3AC
:108430006346ADE70021E4E71A1D9A429B412E00F6
:108440005B42D2080DE751075202120BD9E7C04632
:10845000FF03000002FCFFFFFF0700001E040000F6
:108460003E040000F0B557464E464546DE46E0B5B0
:108470000D0004001F000B03190B160087B06B00E2
:10848000EA0F89469246009401955B0D00D1B7E151
:10849000D54A934200D11DE1C900420F0A43802111
:1084A00009041143C2009046D04A89469B189B4656
:1084B0000023002502933C037A00FB0F3000240BBD
:1084C000520D009300D170E1C74B9A4200D155E1A3
:1084D000DC46C64BD2189444E3460A2D00DD0AE17F
:1084E000730FE4001C4380231B042343F000524617
:1084F000009900264A409246022D11DD0122AA4031
:10850000A6211400C9000C400A4200D0F3E09021DB
:1085100089000A4200D0C4E18821114200D0E5E080
:1085200041460C0C0904020C090C0F001500000454
:10853000000C654347430395B8462F000D00060025
:108540005543AC46454666432D0CB4446544AE42A3
:1085500004D93E0080277F02F619039647463F0460
:108560003F0C2E0C2D04ED1904951D0C1B041B0C47
:1085700000934B431F00009B694363439C463B0CA5
:108580006144C9186C438C4502D980235B02E4180E
:108590003F040B0C3F0C0904C919E4187318059328
:1085A0004B461E04360C1F0C330043439C463B00D5
:1085B000534302936346784372431B0C1218D2183C
:1085C000904204D9802302985B02C0180290029B5B
:1085D000100C1B180293634618043300000C12049D
:1085E000121800986E4343439C46030060467B4349
:1085F0006F43F618050CAD19AB4202D980235B021C
:10860000FF18039B059E2804F61863468E42894195
:108610001B041B0CC3181B19494258188446B61872
:10862000A3429B418C45894196429241029849421E
:10863000604400905B4252420B43009C02998018B8
:10864000904292418C4289412D0C494252420A4348
:108650005B199B18DB19C20D5B0204991A43914602
:1086600072020A43511E8A41F60D1643310042023E
:10867000114308008846DB0156D45A465C4BD21899
:10868000002A00DC13E14B0716D00F215B460140A6
:10869000042911D04146081D40458941CC46494234
:1086A0008C44E14680464846C10105D5514A1040F8
:1086B00080228146D2009A184F4B9A4200DD25E174
:1086C000494643464C07DB081C4352054B021B0B33
:1086D000520D1BE00A0000990A43904600D0DAE0F0
:1086E0009B460223914608250293E4E6009A9946A8
:1086F000924680460296029B022B00D106E1032B94
:1087000033D0012B1AD100220023002412051A4372
:108710005346DB071A432000110007B0F0BCBB46EC
:10872000B246A946A046F0BD01224B080A40494680
:108730001343CA07134398464B08994680215A466B
:10874000C900531C5218002A00DCB1E04046410722
:10875000A9D00F21014004299CD1A4E70F2D00D1FD
:10876000F7E0009BA1469A46804680234A461B03B9
:1087700013431B0344461C4A1B0BC7E759463300EF
:10878000194E234389198B46002B72D102212943AC
:108790000A29B0DC5046009C60408246002D00D182
:1087A00007E10D0000200226A8E62300334351D044
:1087B000002C00D1BEE0200000F01AFA02000B38B5
:1087C0001D231B1A3000D840110003003000083967
:1087D0008C408840234359468A1A084952189346C8
:1087E0000A2D00DC83E686E7FF07000001FCFFFF9F
:1087F000FF030000FFFFFFFEFE0700000DFCFFFF70
:108800000A000B0000990A4390461CD0002B00D1AF
:1088100080E0180000F0ECF902000B381D231B1A51
:10882000009811004D46D84008398D4003002B4375
:108830009946009B8B409846624B00259B1A9B46AD
:108840000023029337E6002399469B460133042513
:10885000029330E6012215430A2D00DD4BE7524614
:1088600000994A409246022D00DC4CE70020012688
:1088700044E603231D430A2D00DD6FE75346009AAB
:10888000882153400122AA409A4603262300114220
:1088900000D145E62AE79B46032380460C25029338
:1088A00009E600239A468023474A1B032EE75B46CE
:1088B0001100373100DA26E711001E3158DA484638
:1088C0001F2104004942891ACC4021001F3205D0E3
:1088D0003E4A9B1898404246024390464246531EE9
:1088E0009A410A4307210C0000231440114209D089
:1088F0000831114004295FD0111D9142A4410A00A2
:1089000064426407D20814430022FFE600230024D7
:108910002D4AFBE600F06CF902000300153020320E
:108920001C2800DC7AE7002188460099083B994022
:10893000894681E700F05CF902000300153020321F
:108940001C2800DC3CE73100083B994000200B006C
:1089500041E780234A461B031A4200D105E71C4227
:1089600000D002E7009A234392460400164ACDE65F
:108970000121891A164A48469B1842469840CA4027
:10898000104342469A40531E9A414B460243CB4005
:10899000510708D00F211140042904D0111D914224
:1089A00092419B1A0A00190208D5012200230024D3
:1089B000ACE600230024A9E60024A3E75C075B02E1
:1089C0001B0B9FE70DFCFFFFFF0700003E040000AC
:1089D0001E040000F0B505000020144C0A034B00F3
:1089E000C90F0F008446120B5B0DA34205DD104C2E
:1089F000A34204DD0F4BC9188C466046F0BD8024AD
:108A0000640322430C4CA34207DCE41AE2405342C5
:108A10009C46002FF1D19446EFE7280007495918EA
:108A20008A400749CB1AD8400243F0E7FE03000012
:108A30001D040000FFFFFF7F13040000EDFBFFFF9C
:108A40003304000070B542024300C40FFE201B0E29
:108A5000591C550A08420BD0E02189006D07120B02
:108A60005B181B051343E40723432800190070BD5E
:108A7000002B14D1002D1BD0280000F0B9F80A28D3
:108A80001CDC0B232A001B1ADA40030015339D401F
:108A90000D4B12031B1A5B05120B5B0DE1E7002D5A
:108AA00009D0130B802212031A436D07074BD8E736
:108AB00000230022D5E70022044BD2E703002A005E
:108AC0000B3B9A400025E3E789030000FF07000005
:108AD00070B50D036D0A4B00440F2C435B0D404DE8
:108AE000A44682B05C1C00900191CA0FC6002C42C3
:108AF0000BD03C495C18FE2C15DDFF200023C0057F
:108B00001843D207104302B070BD604631000143E4
:108B10000020002BF3D00029EFD080236146DB0337
:108B2000FF200B43EBE7002C0DDD009B710F9B0139
:108B3000581E83416046C00003430B43590720D1B0
:108B4000DB08E0B2DBE72100173129DB802160463A
:108B500009040143601C26DB23481D181E20330036
:108B6000AE40001BC3403000A940441EA041014359
:108B70000B430721180008400B4227D19B015B0AD9
:108B8000BDE70F211940042903D19B015B0AE0B224
:108B9000B5E704335901F8D5601C0023C0B2AEE735
:108BA00000200023ABE702200D004042001BC5401F
:108BB0002800023405D00D4C1B19994033000B439B
:108BC0001E003300591E8B410343D2E70F210024BE
:108BD00019400429DDD19B0120005B0A8FE7C046C4
:108BE000FE07000080FCFFFF82FCFFFFA2FCFFFFEE
:108BF0001C2101231B04984201D3000C10391B0ACD
:108C0000984201D3000A08391B09984201D3000990
:108C1000043902A2105C40187047C04604030202E7
:108C200001010101000000000000000010B500215A
:108C3000040000F0A3FB044B1B68002B00D09847F6
:108C4000200001F041FEC046F412002010B5034A96
:108C50000349044800F0DAF810BDC0466001002066
:108C6000199A00007001002041680B4B10B50400F8
:108C7000994201D000F0D0FEA168084B994202D081
:108C8000200000F0C9FEE168054B994202D02000A7
:108C900000F0C2FE10BDC046BC110020241200200E
:108CA0008C120020F0B53A4C3A4B3B4A200083B07E
:108CB00000251A600423082200215C30E36025604F
:108CC0006560A560656625616561A56100F000FAD3
:108CD0002000324F324E334B3349583000932362D9
:108CE00001916162E461A762E66200F0AFFACC2311
:108CF000E5502E4B20006367802308220021C430FA
:108D0000E550A566E5662567A567E56700F0E0F92B
:108D10002200842320006832E250009A0199043333
:108D2000E2500433E1500433E750C0300433E650DE
:108D300000F08CFAD0232000E5500433E5500433D2
:108D4000E5501B4A5C33E550583BE2500433E55094
:108D50002D300433E550082204330021FF30E55064
:108D600000F0B6F92000EC23D030E0502000009A4B
:108D700001990433E2500433E15029300433E750C1
:108D8000FF300433E65000F061FA03B0F0BDC04696
:108D9000BC110020F41200204D8C0000958F0000C3
:108DA000C18F00002D8F0000558F000009000100C9
:108DB0001200020070B50500094C200000F04AFACC
:108DC0006B6B002B05D1074B6B63074B1B68002BAC
:108DD00003D0200000F040FA70BDFFF763FFF8E712
:108DE00000130020698C0000F412002010B5024826
:108DF00000F030FA10BDC0460013002010B5024844
:108E000000F02AFA10BDC04600130020F8B547460E
:108E1000CE46884680B58146170000267D68013D14
:108E20000ED4BC68A389012B07D90E22A35E01339F
:108E300003D021004846C04706436834013DF1D2C3
:108E40003F68002FEAD13000C0BCB946B046F8BD3B
:108E500030B5050089B008000C0000F053FA04ABEF
:108E60002B4A019302230692012202936B6B059019
:108E7000013004940792AC680390002B40D00C2181
:108E8000625E0121636E19421DD0900425D48021B9
:108E900089010A43A2811F4A134063669A0433D4AE
:108EA000280001AA210000F0F9FE421E90410A2587
:108EB0004042636E0543DB0702D4A3899B0512D5AC
:108EC000280009B030BD900511D59004DFD55B13A3
:108ED0001942E5D001256D42EFE75B131942DFD05F
:108EE00001256D42ECE7A06D00F0B6F9E8E7A06D52
:108EF00000F0B0F90C23E25E636E9104CED4C6E7B5
:108F00002800FFF757FFBAE701256D42D3E7C046B7
:108F1000E8AB0000FFDFFFFF10B5034B010018684E
:108F2000FFF796FF10BDC0466C01002070B50C0025
:108F30000E25495F00F038F9002803DB236D1B186C
:108F4000236570BDA389024A1340A381F9E7C04697
:108F5000FFEFFFFFF8B516001F000C228B5E050027
:108F60000C00DA050AD40A4A28001340A381320013
:108F70000E23E15E3B0000F02BF9F8BD00220E232A
:108F8000C95E022300F0FCF80C22A35EEBE7C046AA
:108F9000FFEFFFFF70B50C000E25495F00F0F0F801
:108FA0000C22A35E421C05D080225201134320658F
:108FB000A38170BD014A1340FAE7C046FFEFFFFFEF
:108FC00010B50E23C95E00F0C9F810BDF0B5C64655
:108FD0000D00160000B5884212D9891881420FD9B8
:108FE0008418032A56D8731E002E06D0DA43891837
:108FF000A418CA5CE254013BFBD280BCB846F0BD69
:10900000032E0BD80400711E002EF6D00023013170
:10901000EA5CE25401339942FAD1EEE703242A00D4
:109020002100024303001140144230D10F2E4BD9CE
:109030001027BC462A003409013C2401A04604192B
:10904000A44414681C6054685C6094689C60D46894
:109050001032DC6010336345F3D10F221C000C2367
:1090600010353240334045441600002BCBD06B58AE
:1090700063500431531A032BF9D803261640920883
:10908000013A920004350434AD18A418BBE704007B
:10909000711EBBE723000B439B0701D0531EA5E7BE
:1090A0002B1F9C461300051F6246D258EA50043B12
:1090B000032BF9D80322B308013B9B00C91AE41A19
:1090C00016400439043C8EE732000400CFE7C04666
:1090D00030B50D001400010083070BD003000322FC
:1090E00004E00D70013C0131134204D00133002C27
:1090F000F7D130BD0300032C22D9FF222A401102F0
:1091000089180A0489180F2C26D922091201D218AD
:10911000196059609960D96010339342F8D10F22D9
:10912000224094460C222240644609D062469208AE
:109130009200D21802C39342FCD103246246144029
:109140001A19002CD5D01D7001339A42D1D01D7050
:1091500001339A42F7D1CCE7A446E7E7002370B584
:10916000064C050008002360FCF7D0FF431C00D02C
:1091700070BD2368002BFBD02B60F9E7B8110020ED
:1091800070B50500080011000022064C22601A008C
:10919000FCF7D3FF431C00D070BD2368002BFBD02D
:1091A0002B60F9E7B811002070B505000800110028
:1091B0000022064C22601A00FCF7F4FD431C00D08C
:1091C00070BD2368002BFBD02B60F9E7B81100209D
:1091D00070B50500080011000022064C22601A003C
:1091E000FCF7C4FD431C00D070BD2368002BFBD0EE
:1091F0002B60F9E7B8110020014B18687047C04692
:109200006C01002070B50D4E0D4DAE4207D000240C
:10921000761BB61008CD01349847A642FAD801F063
:1092200055FB084E084DAE4207D00024761BB61001
:1092300008CD01349847A642FAD870BD88070020AF
:109240008807002090070020880700207047C0464C
:109250007047C0467047C0467047C046F0B5C64626
:109260000D00160000B5032A0DD80400711E002E53
:1092700006D000230131EA5CE25401338B42FAD17B
:1092800080BCB846F0BD032402000A43210003005D
:109290001140144232D1320004000F2E1ED9102783
:1092A000BC462A003409013C2401A0460419A44408
:1092B00054685C6094689C60D468DC601468103208
:1092C0001C6010336345F3D10F221C000C231035B2
:1092D0003240334045441600002BC7D06B586350D2
:1092E0000431531A032BF9D8032616409208013A89
:1092F000920004350434AD18A418B7E70400711EB9
:10930000B7E7C046030084469B070BD00300032148
:1093100002E001330B4206D01A78002AF9D16246E6
:10932000981A7047030019680C4A0D488A188A4336
:1093300002420FD15968094A04338A188A4302420B
:1093400008D15968054A04338A188A430242F1D089
:1093500000E001331A78002AFBD1E0E7FFFEFEFEB1
:1093600080808080034B10B5002B02D0024800F0B3
:1093700089F810BD0000000095A00000F0B5DE46A1
:1093800057464E464546E0B53C4B85B003901868BD
:1093900099460091FFF75EFF394B9B461B689A4642
:1093A000002B1FD053465A68541E1BD457461D1D10
:1093B0005E1DC42392008437BF18B84657465B0031
:1093C000FF365344AD18B6180293009B002B15D0FE
:1093D0004246336800998B420FD0043D043A043E64
:1093E000013CF6D24B461868FFF736FF05B0F0BCDB
:1093F000BB46B246A946A046F0BD90462B689A46A9
:109400007B68013BA34230D000232B605346002BE6
:1094100018D07B6801934B461868FFF71DFF0123A6
:10942000A340029A12681A4214D1D0474B461868DA
:10943000FFF710FF5B4601991A687B688B4219D1D0
:10944000BA4217D104235B42043D9844F618013C0C
:10945000BBD2C7E7424611683A008D32FF3212682C
:109460001A4204D10398D047E0E77C60CEE70800B9
:10947000D047DBE7002AB5D0924693E7700300207F
:109480000413002010B5010000230022002000F08A
:109490005BFE10BDF0B54E46DE46574645460C0015
:1094A000E0B50B34814685B0162C21D8102900D99F
:1094B000D0E000F0A1FA102418230221C94DEB18C6
:1094C0001A005F68083A974200D172E103227B6874
:1094D000B9689343FA68CA6091600121FB185A6821
:1094E00048460A435A6000F08FFA38000830B5E069
:1094F00007239C4300D5ADE0A14200D9AAE000F0CB
:109500007BFAFC235B009C4200D2B9E1610A00D1E6
:10951000ABE0042900D980E138239C46A1098C44A2
:10952000E0463931CB00082252429446AD4DEB184B
:109530009C446346DF68BC4512D00B00032661469D
:109540009C4607E0F868002A00DB2CE1814200D14C
:109550002DE107007B68B3431A1B0F2AF2DD414659
:109560002A002F690832974200D10BE103207B6863
:109570008343181B0F2800DD86E12A616A610028F9
:10958000ABDA6A68944680229200934200D316E1D7
:10959000DA08580901238340604618438446D30003
:1095A0005B199A686860FB60BA609F60D7600120B1
:1095B0008B10984060455FD8634603420AD103236D
:1095C0009943634640000431034203D14000043113
:1095D0000342FBD00323A8469C4683460D00E800C7
:1095E00040440600AA46F3680BE061465A688A4385
:1095F000171B1900DB680F2F00DD1BE1002F00DBBC
:109600002FE19E42F1D1534601339A4608369B071B
:10961000E9D1032205E003680838013D834200D008
:10962000E2E12A42F7D14246594653688B435360E0
:109630005A46520093469A421DD8002A06D11AE093
:109640005246043292465A46520093461342F7D08D
:109650005546C4E70C234A461360002005B0F0BC11
:10966000BB46B246A946A046F0BD80233F2240211A
:1096700090469B0057E745460322AF687B689343BB
:109680009A46A34202D31B1B0F2B7EDC564B0820AD
:109690001B6810331E1900F011FD544B83460193D3
:1096A0001B68013304D0731E1B18424213401E0076
:1096B0003100484600F0DCFC8046431C00D1FDE050
:1096C0005346FB18834200D9F6E0494A11680292DA
:1096D000891911605A46013A834200D139E1019853
:1096E0000068013000D13FE14046C31A5B1802997F
:1096F0000B6041460723080018400190194200D131
:10970000F9E0C446310001331B1A9C4461440391C3
:109710005B4411405B1A1A4011004846E0461600AF
:1097200000F0A6FC431C00D13AE1029B196889199C
:1097300019604346C21A012092190243AB605A6075
:10974000AF4213D053460F2B00D811E107220C3B38
:1097500093437A68024005201A437A60FA185060F1
:1097600090600F2B00D921E143465A68214B1868BD
:10977000884200D21960204B1868884200D21960D4
:1097800047469DE06B689C4611E701222100134388
:1097900011433C1979604846AC60636000F034F9CD
:1097A000380008305AE7BA68D060826095E66146B2
:1097B000D6E6DF680231BB4200D1D1E686E65A0A1E
:1097C000042A73D9142A00D9A7E010005C325B3058
:1097D000D200AA18083A160092688846964210D11C
:1097E00081E0C0468003002038130020740300206D
:1097F0000813002034130020301300209268964292
:1098000004D00321506888439842F7D84146D6686F
:10981000FE60BA60B760D760C9E614295CD95429E4
:1098200000D982E06E239C46210B8C446F31E046C8
:10983000CB0078E601200E00454609190443746008
:10984000B4680835E36038439C60A960E96048600B
:10985000CD6048468D60B75000F0D6F83000083033
:10986000FCE601200C008A1851680834014351605D
:1098700022684846D3609A6000F0C6F82000EDE602
:109880002300E108083319E60126391934437C60C6
:1098900029616961CA608A60320002434A60F850F7
:1098A000484600F0B1F838000830D7E69A091000B1
:1098B00039323830D2008CE7AF4242D0AF687A6894
:1098C00003239A43131BA24202D30F2B00DD5CE754
:1098D000484600F099F8C0E65B239C468C445C3116
:1098E000E046CB001FE6012380108340604618430A
:1098F000844668608CE73300594643440193134023
:10990000CB1A1A4011004846160000F0B1FB431C68
:1099100000D00AE70026019807E7542A2BD81A0B33
:1099200010006F326E30D20053E7AA235B009942D9
:109930002BD8DD3B9C46E10B8C447831E046CB00D4
:10994000F1E52B4A11680292891911605A46013AD1
:10995000C5E6104200D0C2E652460123A86892191B
:109960001A438046426001E74146019B1960C0E608
:1099700043465860ACE7AA204000824221D8DA0B67
:10998000100078327730D20023E71A4B994221D861
:109990007C239C46A10C8C447D31E046CB00C2E583
:1099A0000198039B083800261818BEE6390048467F
:1099B000083100F06BFC029B1968AB6898465A6846
:1099C000D4E60C4882420BD89A0C10007D327C30D1
:1099D000D200FEE6FE237E227F2190469B00A2E578
:1099E000FE227E209200F4E643465B6820E6C046F5
:1099F000081300205405000010B50248FFF72AFCA8
:109A000010BDC046F812002010B50248FFF724FC34
:109A100010BDC046F812002070B505000C1E42D0E3
:109A2000002802D0436B002B49D0FFF7DFF901215A
:109A30000C22A35E626E0A4231D19B0542D5210001
:109A4000280000F053F8E36A0600002B04D0280039
:109A5000E1699847002828DBA3891B062AD4216BDB
:109A6000002908D023004033994202D0280000F09A
:109A70000DFC00232363616C002904D0280000F052
:109A800005FC002363640023A381636EDB0728D5F4
:109A9000A06DFFF7DDFBFFF7B1F9300070BD002BC3
:109AA000CDD1FFF7ABF90026F7E70126A38976426F
:109AB0001B06D4D52800216900F0E8FBCFE7FFF7AB
:109AC00079F9B2E7A06DFFF7C5FB0C22A35E002B6E
:109AD000B5D10122636E1342E3D1A06DFFF7BCFB49
:109AE000DFE7A06DFFF7B8FBD2E7C046F0B5C6468A
:109AF00000B50C228B5E80460C001A0754D48021DE
:109B0000626809011943A181002A00DC6DE0A56AA1
:109B1000002D45D042464046166800220260DB0414
:109B200068D400220123E169A8470200431C00D148
:109B30006DE00C23E15EA56A490706D56368D21A79
:109B4000236B002B01D0E36BD21A0023E16940465E
:109B5000A8470C23E15E431C4ED143461A681D2AD8
:109B600061D8324BD340DB075DD5314B0B40A3812D
:109B70000023636023692360C90403D543461B683F
:109B8000002B42D04346216B1E60002908D02300E1
:109B90004033994202D0404600F078FB0023236313
:109BA000002080BCB846F0BD0E69002EF8D00D68CC
:109BB0000022AD1B0E609B0700D14A69A260002DF8
:109BC00004DCEDE736182D1A002DE9DD2B003200FC
:109BD0004046E169676AB8470028F3DC4022A38960
:109BE00013430120A3814042DBE7E26B002A00DD42
:109BF0008DE7D5E7226D9FE70D4B0B40A381002336
:109C0000636023692360C904BCD52065BAE7434675
:109C10001B68002B00D18CE71D2B01D0162BDDD14A
:109C200043461E60BCE740230B43DAE701004020B7
:109C3000FFF7FFFF70B505000C00002802D0436B52
:109C4000002B27D00C22A35E002B11D0626ED2070E
:109C500001D49B050ED528002100FFF747FF636E56
:109C60000500DB0702D4A3899B050FD5280070BD32
:109C70000025FBE7A06DFFF7EDFA28002100FFF7B4
:109C800035FF636E0500DB07F0D4ECE7A06DFFF74E
:109C9000E3FAEBE7FFF78EF8D4E7C046F0B54546A8
:109CA000DE4657464E46E0B5936883B00C009046BA
:109CB0000090002B2AD00C23CA5E13072ED50B6907
:109CC000002B2BD043461E68930734D5B04B00279A
:109CD00000259946002D15D02B004D4500D9AC4BE1
:109CE000626AE169924600983A00D047002800DC99
:109CF000B5E0434642469B681B1A936006D03F1866
:109D00002D1AE9D1376875680836E3E7002003B0FB
:109D1000F0BCBB46B246A946A046F0BD2100009863
:109D200000F03CF9002800D09EE00C23E25E4346A0
:109D30001E689307CAD4D30700D598E0802100237A
:109D4000890000258B4699462368002D4FD059463F
:109D50001800A7680A4255D0BA46AF4200D9DEE0E3
:109D60009021C9000A422ED0606921695F1A430020
:109D70001B18D80FC3185B109A467B1C5B19504602
:109D80000197534501D99A461800520500D4E4E0E2
:109D900001000098FFF77EFB071E00D1F2E0019A58
:109DA0002169FFF75BFAA3897A4A134080221343A3
:109DB000A3815246019B2761F818AA462F00D31AA7
:109DC00020606261A36052464946FFF7FFF84246B1
:109DD0004146A368DB1BA36092682368521B53446F
:109DE00023608A60002A00D190E70C21625E31680E
:109DF000756889460836002DF9D059461800A768BD
:109E00000A42A9D122699A4272D362699246AA4251
:109E10006ED8802328001B069D4200D35E48514621
:109E2000FCF76AFA53464A464343E169676A009879
:109E3000B847002813DD0700434642469B68ED1BE8
:109E4000DB1B936000D161E70C23E25EB944236819
:109E50007BE721000098FFF7EDFE00282BD00C22B5
:109E6000A35E40221343A381012040424FE7002319
:109E70000027B14600209A461E00002F25D000285A
:109E80002BD03300BB469F4200D99B4620682269F5
:109E90006369904203D9A5685D19AB454FDC5B450A
:109EA00040DC656A5246E1690098A847051ED6DD88
:109EB0000120761BCDD0434642469B685B1B9360D6
:109EC00000D123E7AA447F1BD9D14B4608225F6803
:109ED0009144002FF9D01B689A463A000A21504657
:109EE00000F0FAF800284AD053460130C61AC8E7F5
:109EF000AF4200D92F003A0018004946FFF766F834
:109F0000A2682368D21BDB19A2602360002A93D1C8
:109F100021000098FFF78EFE00288DD09FE72F00CC
:109F2000AA4650E75A465146FFF750F85A46A368EA
:109F30005D469B1AA36023685B442360B8E75146E3
:109F40002A00FFF743F8236821005B19009823607B
:109F5000FFF770FE0028ABD081E70200009800F008
:109F60007FFA071E00D024E7009D2169280000F039
:109F70008DF98022A3899343743A2A6071E77B1C90
:109F80001E007FE70C23009A13600C22A35E68E793
:109F900000FCFF7F7FFBFFFFFFFFFF7F334B70B5B0
:109FA000050018680C00002802D0436B002B51D02C
:109FB0000C22A35E1A070FD52269002A16D00C21A5
:109FC000635ED90723D50021A16061690020494261
:109FD000A161002A23D070BDDA063ED55A0724D4E9
:109FE000226908210B43A381002AE8D1A020802107
:109FF000A3898000890003408B42E0D02100280023
:10A0000000F0C2FB0C21635E2269D907DBD400217A
:10A01000980700D461690020A160002ADBD11A06EC
:10A02000D9D540221343A3811CE0216B00290AD01B
:10A0300022004032914204D0280000F027F90C227F
:10A04000A35E0022226324229343002262602269DD
:10A050002260C6E7FEF7AEFEAAE709222A60402288
:10A060001343A38101204042B5E7C0466C010020A4
:10A07000002370B5064C05000800236000F016FCB4
:10A08000431C00D070BD2368002BFBD02B60F9E788
:10A09000B811002070B5074C074D641BA41005D003
:10A0A000013CA300EB589847002CF9D100F014FCB8
:10A0B00070BDC0469407002090070020802310B593
:10A0C0005B01082801D1180010BDFFF795F8162391
:10A0D0000360173BF7E7C0468C4610B5C9B283074B
:10A0E0000CD0032406E003788B4206D00130013AFD
:10A0F000204203D0002AF6D1002010BD032A14D933
:10A100006346FF241C4023021B199C461C04A444E4
:10A110006446036863400A4C1C199C43094B1C426B
:10A1200005D1043A0430032AF2D8002AE4D0821878
:10A1300003788B42E1D001309042F9D1DCE7C04690
:10A14000FFFEFEFE80808080F8B5CE464746204C5C
:10A15000050080B52068160099468846FFF77AF812
:10A160001C4B1A68002A2BD0536820681F2B2ADC4E
:10A17000002D0CD1591C5160414602339B0099506F
:10A18000FFF76AF80020C0BCB946B046F8BD882485
:10A19000990051180E511600873C9C408936FF36B5
:10A1A00037682743376084264F4676008F51022D4B
:10A1B000E0D115008D35FF35296821432960D9E7A5
:10A1C000054A1A60D0E7FFF747F801204042DAE776
:10A1D00070030020041300203C130020F0B5C64695
:10A1E000050000B5804608200C00FFF767FF060059
:10A1F0002800FFF701FC224F3100BB685D68032394
:10A200009D4328001138001B8019FBF7EBFF441E0B
:10A210007443A64207DC00214046FFF729FFBB68D4
:10A220005B19984206D04046FFF7EEFB002080BC49
:10A23000B846F0BD40466142FFF71AFF01300DD02D
:10A2400001222D1BBB6815430E4A5D601368404612
:10A250001B1B1360FFF7D8FB0120E8E700214046F5
:10A26000FFF706FFBA68831A0F2BDCDD064C0549A1
:10A270002468001B086001210B435360D3E7C046EC
:10A28000800300200813002074030020F0B5C646A8
:10A290000C00804600B5002940D0FFF7ADFB21003F
:10A2A00008394E68012533000320AB43CA18944691
:10A2B000526882432800304007006448846864453F
:10A2C00000D171E064466260A41864682C40002FDD
:10A2D00027D10E685E4F891B9B198E68BE4256D0EF
:10A2E000CF68F760BE60002C1DD062461D434D60F4
:10A2F00013608022920093422DD2DA085C09012378
:10A30000A340446823434360D3001B189A68CB6082
:10A310008A609960D1604046FFF776FB80BCB84602
:10A32000F0BD002C0FD19B18624601249268484D65
:10A330001C43CE18AA4259D06546ED68D560AA6084
:10A340004C603360D5E7624635434D601360802230
:10A3500092009342D1D35A0A042A3DD89A09140094
:10A3600039323834D60086193268083E03259642C1
:10A3700003D14CE09268964203D05068A8439842BB
:10A38000F8D8D668CE608A60B160D160C3E7002C8F
:10A3900033D1D218604663468068DB681543C360DA
:10A3A00098604D608A50B6E79A18002F06D10B6866
:10A3B000C91A8C68D218CB68E3609C6001231343F0
:10A3C0004B60244B81601B689342A4D8224B4046CB
:10A3D0001968FFF703FF9EE7142A13D9542A1DD8E2
:10A3E0001A0B14006F326E34D600BCE7D160916056
:10A3F000CA608A604C6033608DE762461D434D60E1
:10A40000136088E714005C325B34D600ABE70123AD
:10A41000A410A340446823434360B3E7AA24640024
:10A42000A24205D8DA0B140078327734D6009AE7C6
:10A430000A4CA24205D89A0C14007D327C34D60016
:10A4400091E7FE267E24B6008DE7C04680030020FB
:10A4500088030020780300203813002054050000F2
:10A46000F0B545464E46DE465746E0B580460D00FF
:10A47000914683B0002900D1A3E04C460B34FFF78E
:10A48000BBFA162C6CD81024A1456CD82F00083FBD
:10A49000796803230E00BB469A469E43A6426DDAB6
:10A4A000B819B84A4368019200939368009A8342AE
:10A4B00000D199E001239A4394468444624652684D
:10A4C0001A4200D072E05346009A9A43B3189C4651
:10A4D0009C424EDD01230B4210D139687B1A59682A
:10A4E000009353469943521893199A469C4200DCB4
:10A4F000C0E073189A469C4200DCBFE049464046E3
:10A50000FEF7C8FF8146002800D10CE15946012220
:10A510004B6893430200CB18083A934200D1D2E033
:10A52000043E242E00D9D3E003002A00132E09D9BB
:10A530002B6803606B6843601B2E00D9CDE00300DD
:10A5400008320833116819605168596092689A603E
:10A5500040462900FFF79AFE4046FFF755FA1DE0F6
:10A5600007239C4390D50C23424613600023994651
:10A5700014E06646C3688268D3609A6001227B68F3
:10A58000311B1340B8190F2920D833437B6043682F
:10A59000134343604046FFF737FAA946484603B0E5
:10A5A000F0BCBB46B246A946A046F0BD01230B4213
:10A5B000A4D15B461A689B1A596800935346994385
:10A5C00097E71100FEF766FF8146E7E73E19234350
:10A5D00011437B607160310043680831134343606D
:10A5E0004046FFF753FED5E7534620009A439319A0
:10A5F00010309C4683427ADAC90700D57EE7396875
:10A600007B1A5968009353469943521893199A46F6
:10A61000984200DD6DE70099CB688A68D3609A6044
:10A620000B00321F08339946242A00D990E0132AE0
:10A6300009D92B688B606B68CB601B2A00D98CE032
:10A6400010310B0008352A681A606A685A60AA68D7
:10A650009A600098019B01199960534601221B1BC7
:10A6600013434B6043681340234343604046FFF766
:10A67000CBF993E7C3688268D3609A6000990F00B2
:10A680008A68CB680837D3609A60321F242A15D8AD
:10A690003B00132A08D92B688B606B68CB601B2AA0
:10A6A00036D810310B0008352A681A606A685A607B
:10A6B000AA689A603D005646009F5FE7290038006F
:10A6C000FEF784FCF6E703225B689343F61855E730
:10A6D00032002900FEF77AFC3AE7AB688360EB684A
:10A6E000C360242E23D00300103210332AE7019BCD
:10A6F00039199960634601221B1B13434B607B6829
:10A700004046134023437B60FFF77EF9A94645E7A7
:10A71000AB6800990B61EB684B61242A0FD00B00EA
:10A7200010351833C0E74046FFF76EF91EE72B6976
:10A7300018320361030069691833416102E72B692C
:10A7400000998B610B006A692033CA611835ABE749
:10A7500029001800FEF73AFC7BE7AB6800990B6113
:10A76000EB684B61242A03D00B00103518336AE7DD
:10A770002B6900998B610B006A692033CA61183517
:10A7800061E7C0468003002070B50C23CA5E050057
:10A790000C0096B0930707D5230043332360236151
:10A7A0000123636116B070BD0E23C95E002931DB41
:10A7B0006A4600F055F800282ADB80212800C900ED
:10A7C000019EFEF767FE0C22A35E00283DD080228A
:10A7D00013438022D2006261F02231001202114044
:10A7E0000A008021A3812060206189018A4234D13E
:10A7F0000E23E15E280000F047F80C22A35E00283B
:10A800002BD003229343012213438022120119E02B
:10A810000C23E25E802313405A425341F0225B42F4
:10A82000920013404033190028001E00FEF732FE4C
:10A830000C22A35E002808D080221343002220604F
:10A84000206166611343A381ACE79A05AAD4032271
:10A85000934302221343A3819EE780221201F1E772
:10A86000002370B5074C0500080011002360FBF7BA
:10A8700055FC431C00D070BD2368002BFBD02B601F
:10A88000F9E7C046B8110020002370B5064C05005A
:10A8900008002360FBF74AFC431C00D070BD23680E
:10A8A000002BFBD02B60F9E7B8110020044A136895
:10A8B000002B03D01818106018007047014BF9E7FF
:10A8C000CC140020D0140020FEE7C046F8B5C046E6
:10A8D000F8BC08BC9E467047F8B5C046F8BC08BC3A
:10A8E0009E46704700C0C101C30302C2C60607C727
:10A8F00005C5C404CC0C0DCD0FCFCE0E0ACACB0BB0
:10A90000C90908C8D81819D91BDBDA1A1EDEDF1FDF
:10A91000DD1D1CDC14D4D515D71716D6D21213D3CF
:10A9200011D1D010F03031F133F3F23236F6F7377F
:10A93000F53534F43CFCFD3DFF3F3EFEFA3A3BFB6F
:10A9400039F9F83828E8E929EB2B2AEAEE2E2FEF1F
:10A950002DEDEC2CE42425E527E7E62622E2E3238F
:10A96000E12120E0A06061A163A3A26266A6A767BF
:10A97000A56564A46CACAD6DAF6F6EAEAA6A6BAB2F
:10A9800069A9A86878B8B979BB7B7ABABE7E7FBF5F
:10A990007DBDBC7CB47475B577B7B67672B2B3734F
:10A9A000B17170B0509091519353529296565797FF
:10A9B000559594549C5C5D9D5F9F9E5E5A9A9B5BEF
:10A9C00099595898884849894B8B8A4A4E8E8F4F9F
:10A9D0008D4D4C8C4484854587474686824243830F
:10A9E0004181804000C1814001C0804101C080415F
:10A9F00000C1814001C0804100C1814000C181404F
:10AA000001C0804101C0804100C1814000C181403E
:10AA100001C0804100C1814001C0804101C080412E
:10AA200000C1814001C0804100C1814000C181401E
:10AA300001C0804100C1814001C0804101C080410E
:10AA400000C1814000C1814001C0804101C08041FE
:10AA500000C1814001C0804100C1814000C18140EE
:10AA600001C0804101C0804100C1814000C18140DE
:10AA700001C0804100C1814001C0804101C08041CE
:10AA800000C1814000C1814001C0804101C08041BE
:10AA900000C1814001C0804100C1814000C18140AE
:10AAA00001C0804100C1814001C0804101C080419E
:10AAB00000C1814001C0804100C1814000C181408E
:10AAC00001C0804101C0804100C1814000C181407E
:10AAD00001C0804100C1814001C0804101C080416E
:10AAE00000C18140040003010303030202000000CF
:10AAF00080000000020408202048617264466175ED
:10AB00006C74210A00000000001BB70000800000E8
:10AB10001027000000000000001BB70000800000AC
:10AB200000000000001BB70002040800606B00007A
:10AB30008C6A0000766A0000F26A0000766A000003
:10AB4000266B0000766A0000F26A00008C6A000042
:10AB50008C6A0000266B0000F26A0000626A000046
:10AB6000626A0000626A0000306B00008C6A0000BC
:10AB70008C6A0000766A0000CE6B0000766A0000E6
:10AB8000266B0000766A0000CE6B00008C6A000025
:10AB90008C6A0000266B0000CE6B0000626A000029
:10ABA000626A0000626A0000C88000007E7F0000C8
:10ABB000F27E00001E7F0000F27E00006080000038
:10ABC000F27E00001E7F00007E7F00007E7F00007E
:10ABD000608000001E7F0000147F0000147F0000D2
:10ABE000147F0000828000000A00000000000000C6
:08ABF0006855FF7F0100000021
:10ABF800640505050505050A00005B02A602F102C9
:10AC08003C038703D40320046B04B80406055205EB
:10AC1800A005ED053C068B06DA0629077807C90763
:10AC280018086808B80808095B09AE09FF09510A3D
:10AC3800A40AF60A490B9D0BF10B450C9A0CEF0C74
:10AC4800440D9A0DF00D470E9E0EF40E4B0FA20FF9
:10AC5800FA0F5310AC1005115F11BA1114126F12CC
:10AC6800CA1225138113DD133A149714F4145215DC
:10AC7800B0150E166C16CB162B178B17EC174D1834
:10AC8800AF1811197319D619391A9D1A011B661BA9
:10AC9800CB1B311C971CFD1C641DCB1D331E9B1E3A
:10ACA800041F6D1FD61F4020AA2015218021EC21EA
:10ACB8005922C6223423A22310248024F124632598
:10ACC800010101010605010005000500030005005A
:10ACD80005000500020002000200320032001E00DA
:10ACE800AB00C3003401B60178009600FA005E019B
:10ACF80067007800C0000701280056007E00AD00FC
:10AD08001C00420066008A00180035004E006800EA
:10AD1800140026003C0056000E001D0031004500BE
:10AD28000C00170026003400E80314054006D0077D
:10AD380020034C047805A406BC02E8031405400669
:10AD480008070200010000000C000000001BB7000B
:10AD58000000000003000000BC110020700100206A
:10AD680000000000BC110020241200208C120020DA
:10AD780000000000000000000000000000000000CB
:10AD880000000000000000000000000000000000BB
:10AD980000000000000000000000000000000000AB
:10ADA800000000000000000000000000000000009B
:10ADB800000000000000000000000000000000008B
:10ADC800000000000000000000000000000000007B
:10ADD800000000000000000000000000000000006B
:10ADE800000000000000000000000000000000005B
:10ADF800000000000000000001000000000000004A
:10AE08000E33CDAB34126DE6ECDE05000B0000000E
:10AE1800000000000000000000000000000000002A
:10AE2800000000000000000000000000000000001A
:10AE3800000000000000000000000000000000000A
:10AE480000000000000000000000000000000000FA
:10AE580000000000000000000000000000000000EA
:10AE680000000000000000000000000000000000DA
:10AE780000000000000000000000000000000000CA
:10AE880000000000000000000000000000000000BA
:10AE980000000000000000000000000000000000AA
:10AEA800000000000000000000000000000000009A
:10AEB800000000000000000000000000000000008A
:10AEC800000000000000000000000000000000007A
:10AED800000000000000000000000000000000006A
:10AEE800000000000000000000000000000000005A
:10AEF800000000000000000000000000000000004A
:10AF08000000000000000000000000000000000039
:10AF18000000000000000000000000000000000029
:10AF28000000000000000000000000000000000019
:10AF38000000000000000000000000000000000009
:10AF480000000000000000000000000000000000F9
:10AF580000000000000000000000000000000000E9
:10AF6800FC120020FFFFFFFF0000020000000000AD
:10AF78000000000000000000800300208003002083
:10AF880088030020880300209003002090030020FD
:10AF98009803002098030020A0030020A0030020AD
:10AFA800A8030020A8030020B0030020B00300205D
:10AFB800B8030020B8030020C0030020C00300200D
:10AFC800C8030020C8030020D0030020D0030020BD
:10AFD800D8030020D8030020E0030020E00300206D
:10AFE800E8030020E8030020F0030020F00300201D
:10AFF800F8030020F80300200004002000040020CB
:10B008000804002008040020100400201004002078
:10B018001804002018040020200400202004002028
:10B0280028040020280400203004002030040020D8
:10B038003804002038040020400400204004002088
:10B048004804002048040020500400205004002038
:10B0580058040020580400206004002060040020E8
:10B068006804002068040020700400207004002098
:10B078007804002078040020800400208004002048
:10B0880088040020880400209004002090040020F8
:10B098009804002098040020A0040020A0040020A8
:10B0A800A8040020A8040020B0040020B004002058
:10B0B800B8040020B8040020C0040020C004002008
:10B0C800C8040020C8040020D0040020D0040020B8
:10B0D800D8040020D8040020E0040020E004002068
:10B0E800E8040020E8040020F0040020F004002018
:10B0F800F8040020F80400200005002000050020C6
:10B108000805002008050020100500201005002073
:10B118001805002018050020200500202005002023
:10B1280028050020280500203005002030050020D3
:10B138003805002038050020400500204005002083
:10B148004805002048050020500500205005002033
:10B1580058050020580500206005002060050020E3
:10B168006805002068050020700500207005002093
:10B178007805002078050020800500208005002043
:10B1880088050020880500209005002090050020F3
:10B198009805002098050020A0050020A0050020A3
:10B1A800A8050020A8050020B0050020B005002053
:10B1B800B8050020B8050020C0050020C005002003
:10B1C800C8050020C8050020D0050020D0050020B3
:10B1D800D8050020D8050020E0050020E005002063
:10B1E800E8050020E8050020F0050020F005002013
:10B1F800F8050020F80500200006002000060020C1
:10B20800080600200806002010060020100600206E
:10B21800180600201806002020060020200600201E
:10B2280028060020280600203006002030060020CE
:10B23800380600203806002040060020400600207E
:10B24800480600204806002050060020500600202E
:10B2580058060020580600206006002060060020DE
:10B26800680600206806002070060020700600208E
:10B27800780600207806002080060020800600203E
:10B2880088060020880600209006002090060020EE
:10B298009806002098060020A0060020A00600209E
:10B2A800A8060020A8060020B0060020B00600204E
:10B2B800B8060020B8060020C0060020C0060020FE
:10B2C800C8060020C8060020D0060020D0060020AE
:10B2D800D8060020D8060020E0060020E00600205E
:10B2E800E8060020E8060020F0060020F00600200E
:10B2F800F8060020F80600200007002000070020BC
:10B308000807002008070020100700201007002069
:10B318001807002018070020200700202007002019
:10B3280028070020280700203007002030070020C9
:10B338003807002038070020400700204007002079
:10B348004807002048070020500700205007002029
:10B3580058070020580700206007002060070020D9
:10B368006807002068070020700700207007002089
:10B378007807002078070020659300003501000059
:04B3880009010000B7
:040000030000614D4B
:00000001FF
